:020000040000FA
:1000000080315428FF3FFF3F7E1480312700931D2D
:1000100012282100101E1228B93136218031270004
:10002000931152282000921C1E282100921C1E2889
:1000300098314C2080312000921052282000111C51
:100040002A282100111C2A28BA31202280312000C0
:10005000111052282000131E36282100131E3628A6
:10006000B031B62080312000131252282000141E17
:1000700052282100141E5228053071127402031CEC
:1000800044283808CC004628CC017116740803199E
:10009000711E4B281412B831D020EE302800990080
:1000A000200014127E10090088310E289D2780310F
:1000B0000F278031C32380312F082200B200200097
:1000C00030082200B300200031082200B40091273C
:1000D00080310F278031C32380312F082200AF00E9
:1000E000200030082200B000200031082200B100BA
:1000F0008B2780310F278031C32380312F082200C6
:10010000AC00200030082200AD00200031082200A1
:10011000AE00972780310F278031C32380312F080D
:100120002200A900200030082200AA002000310887
:100130002200AB009D2780311D278031C3238031F1
:100140002F082300D800200030082300D900200009
:1001500031082300DA00912780311D278031C32325
:1001600080312F082300D500200030082300D6005E
:10017000200031082300D7008B2780311D278031D4
:10018000C32380312F082300D20020003008230031
:10019000D300200031082300D400972780311D2789
:1001A0008031C32380312F082300CF002000300886
:1001B0002300D000200031082300D1008030CC0182
:1001C000CD003F30CE000830C900CF30CA004730E4
:1001D000CB0033302200A600F330A7004030A80047
:1001E000FA011F30FA0A7A020318162B50279631AB
:1001F00094268031AA278031712480313B08C100C8
:100200003C08C2003D08C300502796319426803137
:10021000AA27803171243B08C4003C08C5003D0872
:10022000C60096311D26803141082300C6002000FB
:1002300042082300C700200043082300C800220012
:1002400026082000B400220027082000B500220064
:1002500028082000B6007A089E3153268031963156
:10026000942680312F08B7003008B8003108B90053
:10027000A73120278031031C432923008030C60189
:10028000C7003F30C800230046082000B300230009
:1002900047082000B400230048082000B5002300D0
:1002A00049082000B60023004A082000B7002300B8
:1002B0004B082000B800A6316B268031330823009C
:1002C000C300200034082300C400200035082300A8
:1002D000C5004C082000BB0023004D082000BC00D6
:1002E00023004E082000BD00230043082000BE006C
:1002F000230044082000BF00230045082000C00060
:10030000712480313B082300C30020003C082300F7
:10031000C40020003D082300C5002000630E0339FF
:10032000033A031DCE2921003A087A02031C9D29B5
:100330003D302000C1008A301C2A3A087A02390870
:100340000318B1297A02031CB029230058082000A1
:10035000C100230059082000C20023005A08852A42
:1003600039087A020318C32907307A02031CC3290B
:10037000220032082000C100220033082000C20001
:1003800022003408852A220032082000B200220010
:1003900033082000B30022003408912A630E033989
:1003A000023A031D0E2A21003A087A02031CDD29B5
:1003B00014302000C1006E301C2A3A087A02390835
:1003C0000318F1297A02031CF029230055082000A4
:1003D000C100230056082000C20023005708852AC8
:1003E00039087A020318032A07307A02031C032A09
:1003F00022002F082000C100220030082000C20087
:1004000022003108852A22002F082000B200220095
:1004100030082000B30022003108912A630E03390E
:10042000013A031D502A21003A087A02031C1F2AB0
:10043000AE302000C1000730C2003F30A02A3A0889
:100440007A0239080318332A7A02031C322A23005D
:1004500052082000C100230053082000C2002300DE
:100460005408852A39087A020318452A07307A0287
:10047000031C452A22002C082000C10022002D0860
:100480002000C20022002E08852A22002C0820000D
:10049000B20022002D082000B30022002E08912A6D
:1004A000630E0339031DA62A21003A087A02031CB1
:1004B000602A85302000C1006B30C2003E30A02A87
:1004C0003A087A0239080318742A7A02031C732A3C
:1004D00023004F082000C100230050082000C20064
:1004E00023005108852A39087A020318872A073021
:1004F0007A02031C872A220029082000C10022005A
:100500002A082000C20022002B082000A02A220076
:1005100029082000B20022002A082000B30022008F
:100520002B082000B400CD30AF004C30B0003E307E
:10053000B100C32380312F08C1003008C200310848
:10054000632796311D268031772780312000631F75
:10055000BA2A230065082000C10023006608200095
:10056000C200230067082000632796311D268031D2
:1005700077278031D6278031031DD92A7127803112
:10058000403FAF00413FB000FE268031A32733300B
:10059000C100B330C2003F30C30096311D26803108
:1005A000382780318C24803171272608C03F2708E6
:1005B000C13F803096310B2680315A3A0319E62A22
:1005C0002000C7017A08803EDD26803123004308E1
:1005D0002400A600230044082400A70023004508A7
:1005E0002400A8008C24803171272608C03F2708EA
:1005F000C13F803096310B2680315A3A031DF128D5
:1006000071278031D0277A08803E96310B268031C1
:1006100024003307B50034080318340AB6007127E4
:1006200080313508C03F3608C13FF128D6278031D8
:1006300003194A2B630E0339031D342B2600803027
:10064000DA01DA0ADB0196310B2680315A3A031DB2
:10065000342B9D3096310B26803126005A07DA0064
:100660005B0803185B0ADB0026008030DC01DC0A33
:10067000DD0196310B2680315A3A031D4A2B9E30FC
:1006800096310B26803126005C07DC005D080318DC
:100690005D0ADD0026008030DE01DE0ADF019631D2
:1006A0000B2680315A3A9F30031D612B96310B2661
:1006B000803126005E07DE005F0803185F0ADF0056
:1006C0006C2B96310B268031003A03196C2B2000DD
:1006D0009F30C701DD268031FA010730FA0A7A021D
:1006E0000318852B71278031D027803103303402E5
:1006F000E93003193302031C6D2B7A35203E860046
:10070000E830C03F0330C13F6D2B0F302600A20000
:100710002830A301A4000930A50196310B268031B1
:100720005A3A031D9A2B0A3096310B2680318327C3
:1007300080319D2B9731E027803103302000A700C6
:10074000A801220065352000A9002200660D2000C6
:10075000AA008D313E2528082100D5002000270859
:100760002100D40055082400B400210054082400BE
:10077000B300B436B30C33082100D200240034088F
:100780002100D30008002F08B5003008B60031085A
:10079000B7000310360D370DBA003208B500330824
:1007A000B6003408B7000310360D370DB9003A080B
:1007B0000319E62B39083A0239080318EE2BB50065
:1007C0003A08B50219303502031CED2B3208AF0090
:1007D0003308B0003408B1000800390803190800D4
:1007E0003A0839020318FC2B3A08B5003908B5025B
:1007F00019303502031808000630B800B11BB817CD
:10080000B41B3817B017B101B317B40139083A0255
:100810000318212CB235B30DB40DB90339083A06CB
:1008200003191C2CB8033808073903191C2C0A2C8F
:10083000B136B00CAF0CBA0A3A08390603193B2C92
:10084000182C3A08390203183B2CAF35B00DB10D06
:10085000BA0339083A060319372CB80338080739A0
:100860000319372C252CB436B30CB20CB90A3A084C
:100870003906031D332CB81F462CFF30AF06B006D7
:10088000B106AF0A0319B00A0319B10A381F4E2C7A
:10089000B82780310319B30A0319B40AB8012F0825
:1008A000B2073008B33D3108B43DB41F5E2CB82701
:1008B0000319B30A0319B40AB801B80A3208A70029
:1008C0003308A8003408A9003A08AA003808AB0089
:1008D000A631E2262708AF002808B0002908B10099
:1008E00008003D083C043B040319782C8030BD0609
:1008F0003E08AF003F08B0004008B1003B08B2001E
:100900003C08B3003D08B400C3232F08BB003008E7
:10091000BC003108BD000800B127803103102B0D49
:100920002C0DB2003208031D9A2CA601A701A801C4
:10093000A9010800B12780311730AC36AB0CAA0CE6
:10094000890B9D2C2A08AD00A717A8012608AE0028
:100950002708AF002808B0008E30B101B202B21FE4
:10096000BD2C3208803A8F3E031C952CB136B00C5A
:10097000AF0CAE0CB20FB62CCA2C183032020318D2
:10098000952C32080319CA2CAE35AF0DB00DB10D40
:10099000B203C12C2D080319D82CAE09AF09B00938
:1009A000B109AE0A0319AF0A0319B00A0319B10A53
:1009B0003108A9003008A8002F08A7002E08A600BB
:1009C00008001B3096310B268031013A031D8B2D18
:1009D00020000430C701C70ADD26803120006308EB
:1009E000CF391038E3000630C701DD268031200002
:1009F0000D306313C7000830DD269731D1278031D1
:100A0000E700B931A32180312B2796311D26803193
:100A1000442780311C302000C7000A30DD26803199
:100A200070302200E500E60120000C30C701DD2611
:100A3000803120000A30E811C7000E30DD268031F9
:100A400000302300E2008030E3003F30E400FF305C
:100A50002000C7001130DD268031FF302000C700A4
:100A60001330DD26BB31E9238031031D442DCD3009
:100A70002100A0004C30A1003E30A200CD30A300E8
:100A8000CC30A4003D30552D56080339023A031DE1
:100A9000572D9A302100A0009930A1003F30A200CC
:100AA000CD30A3008C30A4003F30A5005E2D210086
:100AB000A001A101A201A301A401A5010A30200007
:100AC000C7001630DD2680310B302000C7001830FB
:100AD000DD268031FF302000C7008030DD268031E8
:100AE000FF302000C700AA30DD268031FF30200013
:100AF000C700AC30DD268031FF302000C700AE30AB
:100B0000DD26A231A12280315620803120001B3009
:100B1000E411C701DD261C3096310B268031013AE5
:100B2000031DC32DFF302000C7001D30DD2680319E
:100B3000FF302000C7001F30DD268031FF3020004D
:100B4000C7002130DD268031FF302000C700233070
:100B5000DD268031FF302000C7002530DD268031C2
:100B6000FF302000C7002730DD268031FF30200015
:100B7000C7002930DD26BA31F222803120001C3036
:100B80006413C701DD263B3096310B268031013AD4
:100B9000031D662E02302000C7002E30DD26803176
:100BA00050302100ED001E302000C7003030DD261F
:100BB00080311E302100EC0040302000C700323070
:100BC000DD26803140302100E900A03CEA00200011
:100BD0003430C701C70ADD26803121000630EF011D
:100BE000EF0A2000C7003630DD26803106302100B4
:100BF000DD0020003830C701DD2680312000B13013
:100C00005F12C701C70ADD26803120006008F03975
:100C10000138E000B330C701C70ADD26BA310C2223
:100C20008031B530C701DD2680312000B730611139
:100C3000C701C70ADD268031C4278031B930C7011A
:100C4000DD2680312000C1306012C701C70ADD26D1
:100C5000803120006208F0390138E200C330C7015A
:100C6000C70ADD268031BE278031C530C701C70ADB
:100C7000DD268031CA278031C730C701DD268031AB
:100C80002000D3306310C701DD2680312000D5302D
:100C90006311C701C70ADD26803120005E080F39C5
:100CA0001038DE00D730C701C70ADD2680312000AA
:100CB0005F08F0390138DF00D930C701DD26803107
:100CC00020003B30E3116412C701DD264C30963121
:100CD0000B268031013A031D08000F302000C700A9
:100CE0003D30DD2680311E302100DF0020003F3006
:100CF000C701DD268031FC302000DE050430C7004E
:100D00004130DD26803104302100DE0020004330F8
:100D1000C701DD26F9302000E4059631A526803193
:100D20000C30C7005330DD26803102302000C70070
:100D30005530DD26803120004730C701C70ADD2647
:100D40009731AD2780314930C701DD26FC302000C6
:100D5000D505BA31F2228031B631C7268031A331B0
:100D6000EE2380315620A231A122803120004B3069
:100D7000C701DD2680312000FF30E111C70050306F
:100D8000DD268031FF302000C7005130DD2697314D
:100D9000DC278031DD268031FF302000C700733032
:100DA000DD268031FF302000C7007630DD2680311F
:100DB00020004C30E412C701DD2E2000C8003100B5
:100DC0009518DF2E1517200048083100910070306B
:100DD00092009401200047083100930003108B1B00
:100DE00003148B13151555309600AA3096009514F0
:100DF0009518F82E151103188B1708002F08A70057
:100E00003008A8008E30A901AA00AB01A631E22665
:100E10002708AF002808B0002908B1000800B10079
:100E2000210020082000B200210021082000B3008A
:100E3000210022082000B4000800B100210023088E
:100E40002000B200210024082000B3002100250862
:100E50002000B4000800230065082000C40023001F
:100E600066082000C500230067082000C6000800AF
:100E700041082400A600200042082400A70020000A
:100E800043082400A800080041082300E5002000D2
:100E900042082300E600200043082300E700080082
:100EA000220026082000BB00220027082000BC00EA
:100EB000220028082000BD007A08A03E86000130EC
:100EC000870001080800C300230043082000C40075
:100ED000230044082000C500230045082000C60068
:100EE00008007A35203E860003308700080041085C
:100EF0002300C300200042082300C4002000430850
:100F00002300C50008002200E500E601E535E60DF6
:100F1000E535E60D0800AE302000AF000730B00028
:100F20003F3414302000AF006E30B0003F348530C5
:100F30002000AF006B30B0003E343D302000AF00E9
:100F40008A30B0003F342F08C4003008C500310893
:100F5000C60008002F08BE003008BF003108C000DE
:100F600008002608AA002708AB002808AC000800E3
:100F7000FF30B206B306B406B20A080020006208C9
:100F8000CF391038E200080020006108FC39013830
:100F9000E1000800200062083F394038E200080004
:100FA000403F2400B300413FB40008002000550832
:100FB0000339033A0800521908005E080339023A5F
:100FC0000319E82F5E0E0F39013A031D0800F92FAF
:100FD0005E0E0F39013A031D0800541CF62F220043
:100FE0000C19F32F0C150E1C0E14080054180800D1
:100FF000F92F22000C190C110E180E100800FF3FDB
:10100000FF3F003480344034003480343F34663451
:10101000A6343F3401340034FF345F340130FA0029
:1010200031308400A0308500D03086000030870049
:10103000203098310F20883118308400A03085008E
:101040005630860001308700193098310F208831E2
:101050000130840088308500DF3086000130870051
:101060000D3098310F2088314930F001F101F20143
:10107000F301F4018400003085002030983109200C
:101080008831A0308400003085003030983109204C
:1010900088312030840001308500363098310920B5
:1010A0008831A0308400013085003F30983109201C
:1010B000883146308400023085001F309831092085
:1010C0008831A030840002308500403098310920FA
:1010D0008831203084000330850040309831092069
:1010E00088317E102000742821008E01B531BA2588
:1010F0008831721D7E28192288310B292000491C55
:1011000084288731DB2788312000CB1E8C28B72725
:1011100088312100B401B5012C21A0315120883142
:1011200020005F1A9628B2313A228831632588312F
:10113000382688310E21883120004C1EC728073000
:1011400074020318C628F01B7318B928F118B928BF
:10115000353096310B2688315A3A031DB428363083
:1011600096310B268831B52806302100DD00731436
:10117000C728731CC72821005D08031DC728083035
:101180002000E8062100DD01DD0AC72873109B312D
:10119000442388310E2188312C218831F019D4283C
:1011A000C2307402031CD728B3268831F011210005
:1011B0009D1C701BE6289F31552788312F0823007E
:1011C000DC0020002E082300DB0070172000511CDB
:1011D000EC28BA2620005110A531242588310E2193
:1011E00088312100141AF6285A2788312C21883199
:1011F00002302100350259300319340203180B293B
:101200009831B5208831200052190B29FF30250074
:1012100096002000D2100E2188317928F01E18295E
:101220009731F72788319631DB26883172112129D1
:101230002100320F1E29330A03192129B20A03198A
:10124000B30A711F08009731EA27883190310020D6
:1012500088317211BD31332D711420004A19AA2929
:10126000DE199829F01C3629013037290030A800F2
:10127000541C3C2901303D2900302806031942291D
:10128000CD1A5A29F01C4629013047290030A80000
:10129000541C4C2901304D2900302806031D5229C9
:1012A0004D1A5A29033021006706031D6829430897
:1012B000031D6829F01720000A2788310330F11038
:1012C0006706031DAA294308031DAA29F114AA29A8
:1012D00003306706031D782920005B0821004302C4
:1012E000031C75292000CB1EAA292100430895293B
:1012F00002306706031D882920005B082100440294
:10130000031C85292000CB1EAA2921004408952909
:10131000670BAA2920005B0821004502031C9329C2
:101320002000CB1EAA29210045082000DB00AA29A5
:101330002200500BA22920004E18A229F0170A27DC
:101340008831AA292000CD1EA7294E10AA294D1E9A
:10135000AA294E14711CCE2974080319BA29003029
:1013600021002D02F63003192C02031CBA29F53096
:10137000AC00AD0121002C082D04031DCE29F01373
:10138000F1102000CB1ECE2921006708031DCE29B5
:10139000A23096310B2688312000DB00711DE22936
:1013A00022003F084004031DE2292100E701F1105B
:1013B0002000CB1AF01BE229A23096310B2688318F
:1013C0002000DB0020004A19F013F01B721E0A2ACD
:1013D00022003B083C04031D0A2A20005835203E09
:1013E000860003308700403F2200B900413FBA0029
:1013F000200058359E314A268831AB000430200049
:101400005802031CCC15DC302200BB000B30BC00A2
:101410007212D501F01B080072162000CC112200B8
:101420003B083C04031908000130BB020030BC3B00
:1014300008002100AA01AB0120004B10CB1049137A
:10144000CB114B12CA124A1322008E1020004B1DE2
:101450002C2A22000E152E2A22000E118E1174083D
:10146000031D892A20005808031D892A701C3A2A66
:10147000F0143B2AF010701120004C119631D42644
:10148000883120005115F111F013F015F11E4C2A8E
:101490002100921B4C2A921021009213322788318E
:1014A000031D542A5418742A210050085104031DA6
:1014B000742AF01C602A3D002008E0390D38A00095
:1014C000F018672A3D001208E0390D389200AA2270
:1014D00088312000D21C862A22000C110E10E03028
:1014E0003D00A0059205862A2100500851040319E9
:1014F0007E2A0130D0020030D13B862A3227883143
:101500000319541C862A22000C110E10DF22883188
:10151000A72AFF302100D000D10056085704031D30
:101520009C2A9631D4268831200051157408C700B2
:101530000030F8228831F400220063086404031D9F
:10154000A72A7408031DA72A2000D801D9012C005E
:10155000980108002000D218080021003708031D58
:10156000DD2A250016080319B72A9603BC2A160897
:10157000031DBC2A2000D21421005F08B700721995
:10158000D82A9E3169268831031DC92A2100B73621
:10159000D82A9E31A2268831031DD82A2100370877
:1015A0002000A700A736A736270821003702B7007A
:1015B0002000611E08009F31062FB703080020009D
:1015C000CC18ED2AF119080022000C103D00900102
:1015D00022008C103D0091010800F1190800220042
:1015E0000C143D00900122008C143D009101080074
:1015F0002000C800F126883120004D082400330661
:10160000FC3933062000CD00701E112B0330210061
:10161000A800A90120004808031DF42C5527883193
:10162000F42CF01B682C23002308200047024708F5
:101630000318302B480203182F2B4C0E890C03394A
:1016400003192F2B2727883103192F2B4C0E240029
:10165000B300330C0339B300B303FF2688314708C6
:1016600048020318362B21005C083C2B480847022F
:1016700003183E2B21005B08A800A9012000F126D9
:1016800088310230330203187C2B200047084802BF
:1016900003187C2B41278831031D532B21005C0844
:1016A000A8000230642B46278831031D5C2B2100E3
:1016B0005C08A8000430642B3C278831031D692B8B
:1016C00021005C08A8000630A901A8070318A90A90
:1016D000D32B142788313408803AB5008030350286
:1016E000031D762B2000470824003302031CD32B54
:1016F00002302100A800D22B2000F12688310230D0
:1017000033020318D32B2000480847020318D32BB9
:1017100023002808200047020318982B47082300BD
:1017200025020318982B0C302100A800A901CB2B0F
:101730004B278831031DA12B21005B08A800023034
:10174000A92B50278831031DAB2B21005B08A80073
:101750000330A901C82B41278831031DB52BD92699
:101760008831031CA9030430C82B46278831031D88
:10177000BF2BD9268831031CA9030530C82B3C2771
:101780008831031DCB2BD9268831031CA9030630D1
:10179000A8070318A90A372788310318D32B21007B
:1017A000A801A80AA90137278831031C362C27274E
:1017B0008831031DF32B4708230026020318F32B5F
:1017C000210029082400B400210028082400B300C7
:1017D000B436B30C330821002802A80024003408D2
:1017E0002100293BA90020009E31A2268831031D3B
:1017F000072C23002908200047020318012C06307B
:10180000022C0330E626A331D9238831F7262000A5
:10181000B03197208831031D222C23002A08200094
:10182000470203181B2C0C30E626A331D92388313C
:10183000F7268831222C2100A835A90DA835A90D3D
:10184000A835A90D20004C0E890C0339031D362C38
:1018500023002B08200047020318302C1330312CB2
:101860000E30E626A331D9238831F7262100290836
:101870002000B000210028082000AF008631FE269D
:1018800088318731A3278831230062082000C100F6
:10189000230063082000C200230064082000C30066
:1018A00096311D26883187313827883184318C2440
:1018B000883127082100A900240026082100A8005B
:1018C00020004D0803392400B300FF268831E62CA0
:1018D00022003A082100A900220039082100A800AE
:1018E000003022003A02023003193902031CE22CB4
:1018F0002000CC19E22C3C27883103198D2C992C1F
:1019000021005208A8075308E12C1E278831C02C5B
:1019100021005408A8075508E12C56080339013A5C
:101920000319802C033A0319852C013A0319882CDA
:10193000E22C46278831031DA42C220065082100D3
:10194000A80722006608E02C412788310319882C5B
:10195000502788310319882C4B2788310319802C94
:1019600023002608200047060319852C230027089A
:1019700020004706031DC82C1E278831B436B30C3F
:10198000B436B30C33082100A80724003408E02C37
:101990002300280820004706031DE22C0630A7007C
:1019A000A801210053082000AA00210052082000AD
:1019B000A9003E25883127082100A8072000280813
:1019C0002100A93D701DE62C552788313727883125
:1019D000031CF21CF42C2100A801A90120005B08C3
:1019E000031DF42CC701C70A9F310F278831031943
:1019F0003506031D052DEF303302FF300319320287
:101A0000031C052DA801A80AA901200048084702C7
:101A1000031CF01B0D2D701DC70A47084802031C4C
:101A2000C7035908031D362D2C0018082000470253
:101A30000318362D580B362D1427883120004708FF
:101A40002400330634040319F21B362D21004C0EFA
:101A50000F39200047075A07C700F2172100CC01B1
:101A60002000DA012100B8012200CF01210029085D
:101A7000D7002808D600200047080800AB01AC01B9
:101A80002708280403195E2DAD01AD0AA81B4B2DB4
:101A9000A735A80D452DAB35AC0D28082A02031D2E
:101AA000532D27082902031C5A2D2708A9022808AC
:101AB000AA3B2B14A836A70CAD0B4B2D2C08A80065
:101AC0002B08A700080020005E0E0F39013A031D05
:101AD000712D4A1ECA1D6E2D0130C906C8268831D7
:101AE0000C2E5E0E0F39023A031D7B2D4A1ECA1DB5
:101AF0006E2D0430982D5E0E0F39033A031D852D8F
:101B00004A1ECA1D6E2D02306D2D5E0E0F39043A2D
:101B1000031D8F2D4A1ECA1D6E2D04306D2D5E0EC5
:101B20000F39053A031D9A2D4A1ECA1D6E2D02302B
:101B3000CC066E2D5E0E0F39063A031DA72D4A1EE8
:101B4000CA1DA42D2030CA06C8268831002E5E0E7C
:101B50000F39073A031DC62D4A1ECA1DB12D20306C
:101B6000CA06C82688315B080319BC2D22008E11D5
:101B7000A731A82788310C2E7408031D0C2E2100D4
:101B800030083104031D0C2E2000002E5E0E0F398C
:101B9000083A031DE12D4A1ECA1DD02D2030CA0669
:101BA000C82688315B080319DA2DCA1EB62D22001B
:101BB0008E15B82D7408031D0C2E21003008310439
:101BC000082E5E0E0F39093A031DF12D4A1ECA1D5B
:101BD000EB2D2030CA06C8268831F01C5219052E7C
:101BE000002E5E0E0F390A3A031D0C2E4A1ECA1D26
:101BF000FB2D2030CA06C8268831F0185219052E50
:101C0000CA1E0A2E22008E150C2E5E080339023AD7
:101C1000031D0C2E22008E1120004A0E890C013962
:101C20002400B300A93096310B26883124003306F6
:101C30000319232E00302000CA1A0130C700A93032
:101C40008631DD2688312000490801392400B3009F
:101C5000A73096310B26883124003306031908007B
:101C60000030200049180130C700A7308631DD2E32
:101C700020005F080F39013A031D482E2C278831B8
:101C8000A70DA70D4A082706FB392706CA00892E8B
:101C90005F080F39023A031D542E2C278831A70DF7
:101CA0004C082706FD395F2E5F080F39033A031DE4
:101CB000622E2C278831A70E4C082706EF392706FD
:101CC000CC00892E5F080F39043A031D6F2E4A1F7E
:101CD0006C2E2000C914892E2000C910892E5F089F
:101CE0000F39053A031D7C2E4A1F792E2000491515
:101CF000892E20004911892E5F080F39063A031DED
:101D0000892EF11A4A1F872E21009210892E210058
:101D100092142000D21B08005F080F39043A0319FF
:101D2000962E5E0E0F39033A031D9B2EC91C9B2E67
:101D300021000E149D2E21000E1020005F080F3987
:101D4000053A0319A82E5E0E0F39043A031DB02E72
:101D5000491DAD2E21000C15080021000C110800B2
:101D600021000C1108009631D42670172000521063
:101D7000D113080023005C082000C30023005B0887
:101D80002000C200A131E22188310E21A431A12C12
:101D90004A0C2400B300B30C330C0139B400B40E68
:101DA00020004A0824003406EF3934062000CA0017
:101DB000080021005B08A800A90120004C0E890C36
:101DC00003392400B3002100A8020800A700A801DD
:101DD000210029082000AA00210028082000A900CD
:101DE00008004C0E890C03392400B30008002808B1
:101DF0002100A900200027082100A8000800B30E38
:101E0000B30D20004C08240033069F393306200010
:101E1000CC000800DB015808D9004E3071102100B9
:101E2000AC000230AD00080023002108FF3E240072
:101E3000B300FF3003180030B4000800210053083D
:101E40002400B400210052082400B30008004C0E06
:101E5000890C0339033A08004A0E890C890C0139B0
:101E6000A700080020005E080339023A080023009A
:101E7000210820004702080023002108200047060F
:101E8000080023002308200047060800230022083A
:101E90002000470608002300250820004706080008
:101EA0002300240820004706080002302100A80073
:101EB000A901080023002108740203186B2F2000D9
:101EC0005B08031D6B2F5A080319672FDA032100E3
:101ED0004C08031DCC01F119080021004C0820001A
:101EE000AB00AC0174085A07AD00AE01AE0D2B0873
:101EF0002D07AF002C082E3DB000803AB100803095
:101F00003102031D852FC1302F02031C882FB12FF2
:101F1000A03020001E06031D942F0630A700740871
:101F20009631DE268831A42F80301E06031D9F2F98
:101F30000330A70074089631DE268831A42F603064
:101F40001E06031DA62F74367402A72F7408A82F2F
:101F50002100B60020005A0721004C072C009800F1
:101F6000080020001E08023E2C0098000800A03047
:101F700096310B2688315A3A0319080021005A304D
:101F8000CE012000C700A0308631DD268831003028
:101F9000701801302000C700A1308631DD2688315D
:101FA000210048082000C700A2308631DD26883194
:101FB0007F3096310B268831210048060319E72F20
:101FC00048082000C7007F308631DD268831003088
:101FD00020004B180130C700A3308631DD26883140
:101FE000003020004A1B0130C700A5308631DD26B5
:101FF00020004C0E890C0339C700A6308631DD2E37
:1020000021004108031D0E282C082D04031D09285A
:10201000F013200054108C1A541422282000541C51
:102020001328013014280030A7008C1E1928013015
:102030001A28003027060319222821004108031915
:102040002228C1032000541C2728013028280030F2
:10205000A7008C1E2D2801302E2800302706031DD6
:10206000080038302100C1000800210092183A28E9
:10207000A027903111184128200099019A012100D0
:102080001114FF302000C70052308631DD26903118
:10209000DC278631DD26903121000C110E10220044
:1020A0000C110E102000541C5D285E080339023A02
:1020B000031D5D2822000C150E1470162000D21589
:1020C000A331EE239031F1112000491362080F393A
:1020D000013A031974286208F0390138E2003F30F0
:1020E000E205CF30E20563106012E3112000D21D3B
:1020F00053294C0E890C0339013E2100DE0041308A
:102100000B26903121005E0603199B28A52621008D
:102110005E082000C70041308631DD269031403016
:102120000B2690315A3A03199B28B031A9209031DF
:102130008631DD26903120004B1CA2286408F93935
:102140000238A7284A1FA9286408F9390438E4008E
:10215000AB28F930E405640C03392400C000433097
:102160000B269031240040060319C928A526B0315A
:102170009C2090318631DD26903142300B26903103
:102180005A3A0319C928B031AD2090318631DD2685
:102190009031F01ED028F7279031DB269031D928D6
:1021A0002100320FD628330A0319D928B20A03199D
:1021B000B30A711BF11BE028EA27BD3133259031AA
:1021C0009B31442390318F315A2790312000CB1D11
:1021D000102952300B2690315A3A03191029B03188
:1021E000932090318631DD269031200058089E31B1
:1021F00053269031C70053308631DD2690312000C0
:10220000541C09295E080339023A031D09292200DA
:102210000C118F31322790310319102922000C152F
:1022200052300B2690315A3A031D34297408031D8D
:10223000342953300B269031C03C2100D9001F3087
:102240002000A70021005908DE262100D900D90A64
:1022500059082000C70076308631DD269031B6312E
:10226000C72690312000D2114B300B269031003A16
:10227000031D762820005A30D2117012C700523048
:102280008631DD2690315A302000C7005430863127
:10229000DD269031200055080339C700743086319F
:1022A000DD269031762870109D31C725903170124F
:1022B000A331EE239031F401210010124B300B2694
:1022C00090312400C000C00E70084006EF3940066F
:1022D000F00023003E082100C900D601D7012200EA
:1022E0003C30E301E401EC00210092187929A02799
:1022F0009031701E492A2200C701C801983146203A
:102300009031490874060319912956085704031D92
:102310009129D4269E31D42690318A31F8229031E9
:10232000F4008F315A279031210049087406031DAB
:10233000BB2974080319BB291E30FA007A08031957
:10234000BB297A089E31532690317406031DB929A2
:102350007A089F3E860001089F311727903124009C
:10236000C000C101A731682790314008C03F410833
:10237000C13FFA039E297408031D792920005A30B1
:102380004C11F1117012C70050308631DD269031AA
:10239000200056080339C70051308631DD269031C0
:1023A000200055080339C70073308631DD2690318F
:1023B000250040084104031DDF29FF30E0295A3081
:1023C0002000C70054308631DD26903154300B2672
:1023D00090315A3A031D422AFA011E30FA0A7A0253
:1023E00003182E2A7A35A23E860002308700403F2D
:1023F0002400C000413FC1007A35A03E8600403F26
:10240000C200413FC30041084302031D092A40089E
:102410004202031CED29A73168279031403FC000DC
:10242000413FC10000304102FF3003194002031850
:10243000ED297A35A03E8600403FC000413FC100F3
:102440004008013EC2000030413DC3007A35A23E43
:1024500086004208C03F4308C13FED29FA01FA0A4D
:102460001F307A020318422AA731682790310108E9
:102470002000C7007A08543E8631DD269031951839
:10248000302A2F2A20004B30C7018631DD269031BB
:10249000792922000C150E10CF30EC01EC0A200037
:1024A0009B0521001016080001300B2690315A3A86
:1024B000031D742A02300B269031003A0319692A51
:1024C00002300B2690312200EF0064306F02031CB3
:1024D000742A3D302000C70002308631DD2690315D
:1024E000EF278631DD26903101300B2690315A3AA4
:1024F000031D7E2A02300B2690317F2A3D302100B9
:10250000EE0053300B2690312200EF0005306F02B1
:10251000031C932A53300B2690312200EF008130A8
:102520006F02031C9D2AF3278631DD269031B031DE
:10253000932090318631DD269031AD279031FC30EB
:10254000D505A0300B2690315A3A031DA92A200048
:10255000CB1646300B2690315A3A031DB92A473024
:102560000B2690312200EF00200056088C27903176
:10257000BD2A20005608FC390138D60048300B2609
:1025800090315A3A031DCA2A49300B2690317627DA
:102590009031CD2AFC302000D50548300B269031F3
:1025A0005A3A0319EA2A73300B2690312200EF00C1
:1025B00004306F020318EA2A73300B269031762715
:1025C0000339C70049308631DD269031FC2786313A
:1025D000DD26903103300B2690315A3A031DFB2A39
:1025E00004300B2690312200EF00EF0E200063082C
:1025F000C0279031FD2AE5279031E30005300B26F6
:1026000090315A3A031D112B06300B2690312200CF
:10261000EF00EF0E92279031BF396F062000E300E4
:10262000132B2000631307300B2690315A3A031DF9
:10263000212B08300B269031942690316B27903156
:10264000222BD127E700B931A321903187312B27E5
:1026500090311D2687314427903109300B26903167
:102660005A3A031D392B0A300B26873183279031C4
:102670003B2BE02790310B300B2690315A3A031D4B
:102680004B2B0C300B269031992790316808A727E7
:102690009031E8004D2B2000E8110D300B269031D1
:1026A0005A3A031D5B2B0E300B2690319426903145
:1026B00081279031602B23002030E201E30041307C
:1026C000E400B931A32190312E2790311D2690319D
:1026D0005327903111300B2690315A3A031D802B2D
:1026E00012300B269031942690312F082100A00043
:1026F000200030082100A100200031082100962B85
:10270000BB31E9239031031D8B2B00302100A00049
:10271000A1004030962B56080339023A031D982B2E
:1027200000302100A0004030A1004130A2009C2BCD
:102730002100A001A101A20113300B2690315A3AC9
:10274000031DB22B14300B269031942690312F08A4
:102750002100A300200030082100A400200031083F
:102760002100C72BBB31E9239031031DBD2B210074
:102770008030A301A4003F30C72B56080339023A2A
:10278000031DC92B21003030A301A4004130A50056
:10279000CD2B2100A301A401A501B931A3219031C2
:1027A000142790311D2690313B27B931A321903158
:1027B000212790311D2690314727903115300B2667
:1027C00090315A3A031DE82B16300B269031E92B35
:1027D0000A302100DC0017300B2690315A3A031DD5
:1027E000F52B18300B269031F62B0B302100DB0037
:1027F000AA300B2690315A3A031D022CAB300B261F
:102800009031032C14302100C500AC300B269031E0
:102810005A3A031D0F2CAD300B269031102C0F307F
:102820002100C400AE300B2690315A3A031D1C2CF7
:10283000AF300B2690311D2C0A302100C300200040
:102840005508CB279031031C282CFC302000D505DF
:1028500020005608CB279031031C2F2CAD27BA310E
:10286000F22290312D300B2690315A3A031D462C1E
:102870002E300B269031013A031D402C2830572C66
:102880002E300B269031023A031D482C5030572C25
:102890002E300B269031033A031D502C8030572CDC
:1028A0002E300B269031043A031D592CA030210004
:1028B000ED002F300B2690315A3A031D632C303037
:1028C0000B269031642C1E302100EC0031300B2699
:1028D00090315A3A031D702C32300B269031712CF6
:1028E00040302100E900A03CEA0033300B26903153
:1028F0005A3A031D7F2C34300B269031802C023045
:102900002100EF0035300B2690315A3A031D8C2CF4
:1029100036300B2690318D2C06302100DD0037300B
:102920000B2690315A3A031DA12C38300B269031DA
:102930002200EF00EF0E20005F08D6279031DF0065
:10294000A32C20005F125F1EA82C491722008E14B2
:102950003C300B2690315A3A031DB32C3D300B26E8
:1029600090310907B42C1E302100DF000A305F02CD
:102970000318BD2C20006116BF2C200061123E30D0
:102980000B2690315A3A031DD02C3F300B26903144
:102990002200EF0020005E088C279031DE00D32C4F
:1029A000FC302000DE054A300B2690312200EF007B
:1029B00002306F020318E62C4A300B26903199271B
:1029C00090315E08A7279031DE00E82C2000DE1150
:1029D000B0300B2690315A3A031DF82CB1300B263B
:1029E00090312200EF0020006008B3279031FC2CCA
:1029F00020006008F0390138E000B2300B26903139
:102A00005A3A031D122DB3300B2690312200EF00ED
:102A1000EF0EEF0D2000600822006F069F396F0651
:102A20002000162D200060089F392038E000B430C7
:102A30000B2690315A3A031D2D2DB5300B269031BF
:102A40002200EF00EF0DEF0D2000610822006F065D
:102A5000FB396F062000E1002F2D20006111B630F8
:102A60000B2690315A3A031D3F2DB7300B2690317B
:102A70002200EF00200061088C279031432D2000B8
:102A80006108FC390138E100B8300B2690315A3A20
:102A9000031D562DB9300B2690312200EF00EF0EAA
:102AA00020006008D6279031E000582D20006012E9
:102AB000C0300B2690315A3A031D682DC1300B26C9
:102AC00090312200EF0020006208B32790316C2D76
:102AD00020006208F0390138E200C2300B26903144
:102AE0005A3A031D7E2DC3300B2690312200EF0091
:102AF000EF0E20006208C0279031822D200062086E
:102B0000CF391038E200C4300B2690315A3A031DF9
:102B1000992DC5300B2690312200EF00EF0EEF0DFE
:102B2000EF0D2000620822006F063F396F0620007B
:102B30009D2D200062083F394038E200C6300B2648
:102B400090315A3A031DB22DC7300B269031220026
:102B5000EF002000630822006F06FE396F06200098
:102B6000E300B42D20006310D2300B2690315A3A86
:102B7000031DC62DD3300B2690312200EF00922783
:102B80009031FB396F062000E300C82D200063114F
:102B9000D4300B2690315A3A031DDC2DD5300B264C
:102BA00090312200EF00EF0E20005E0822006F0639
:102BB0000F396F062000E02D20005E080F39103815
:102BC000DE00D6300B2690315A3A031DF12DD73056
:102BD0000B2690312200EF0020005F08B3279031D0
:102BE000F52D20005F08F0390138DF00D8300B26C2
:102BF00090315A3A031D082ED9300B26903122000D
:102C0000EF00EF0D9227F7396F062000E300080070
:102C10002000E31108002000A7000F2E2000640010
:102C2000310095180E2E151720002708310091004D
:102C30007030920015141308080041082300EC00BE
:102C4000200042082300ED0020004308B9279031FE
:102C5000A0002008031D2D2EC62F200044082300AD
:102C6000EC00200045082300ED0020004608B927AD
:102C70009031A5002508031D3E2EC62F25087B3E5A
:102C8000A007200043082400A500200046082400D7
:102C9000A5068030A5052000FF30C217C517C40562
:102CA000C505C60124000730A101A201A301A400AB
:102CB0002000411C5D2E5F2790312000C336C20CDE
:102CC000C10CC435C50DC60D2400A40B582E093007
:102CD000A4002000411C6E2E5F2790312000C336D7
:102CE000C20CC10C2400A336A20CA10CA40B692EAB
:102CF00021082000A700240022082000A8002400AA
:102D000023082000A900240020082000AA00240095
:102D100025082000AB00A631E2262708C1002808BC
:102D2000C2002908C30008002000B300A7008E30AD
:102D3000A801A901AA00AB01A631E2262708AF002D
:102D40002808B0002908B1000800200091101F15C4
:102D5000FC309F05640C0339013A031DB42E1F0893
:102D6000FC3901389F00BB2E640C0339023A031D65
:102D7000BB2E03309F0487309F05C0309E00033078
:102D800021005E06031DC62EA030CF2E02305E0647
:102D9000031DCC2E8030CF2E5E0BD12E6030200054
:102DA0009E0020009D0108002300DD01DE012200BD
:102DB000CB01CA010800F726B031E6282000A800A0
:102DC000AA0127080319F52EA901A90AA71BEA2EB3
:102DD000A735E52EAA3527082802031CF22E27085E
:102DE000A8022A14A736A90BEA2E2A0808002430C4
:102DF0004002031C012F413040020318012F3F14F1
:102E000008000F304002031C0B2F1E304002031835
:102E10000B2F3F1008006F304002031C0800BE302B
:102E20004002031CBF140800210020082000C40039
:102E3000210021082000C500210022082000C60032
:102E40000800210023082000C400210024082000DD
:102E5000C500210025082000C600080023006208E4
:102E60002000C400230063082000C500230064087C
:102E70002000C600080041082100A00020004208F0
:102E80002100A100200043082100A2000800410801
:102E90002100A300200042082100A40020004308D4
:102EA0002100A500080041082300E200200042089C
:102EB0002300E300200043082300E4000800440846
:102EC0002400A107200045082400A23D2000460858
:102ED0002400A33D08002F082300E500200030084F
:102EE0002300E60020003108230008002200EF0044
:102EF0002000550822006F06FC396F062000D5001F
:102F000008002F082300E200200030082300E3001F
:102F1000200031082300080022006F06FC396F06EC
:102F200020000800EF0DEF0D2000630822006F065F
:102F300008002200EF00EF0DEF0DEF0D200008005C
:102F400028009501FF30960021009214080022000D
:102F50006F06F7396F062000080020005608FC397C
:102F60000138D600080022006F06F0396F062000F5
:102F700008002300EE0003106D0D6E0D2400080004
:102F800022006F06CF396F06200008002000C10123
:102F9000C201C301080003392200EF0004306F02B0
:102FA000080023005030E501E600413422006F069E
:102FB000EF396F0620000800FF302000C7005434AE
:102FC00070302200E500E601080020006308CF39D8
:102FD0001038080071132200C701C80108005A30D8
:102FE0002000C70001340C302000C70053342100FA
:102FF000B201B301F01208005A302000C700483473
:10300000FF3FFF3FFF3FFF3FFF3FFF3FFF3FFF3FD0
:10301000FF3F640080010131890B0A280034FE0063
:1030200012001E00FE0B1028003420005D08210055
:10303000CF003F30CF05F31C1F283D30CF074F088E
:103040006E06031D26282000CB1E332821004F08C2
:103050006E06031D3E282000CB1E3E284030210076
:103060004E02031C3E2820005415CB1246209831F6
:103070002200C701C801412072110800200054112C
:103080000800F11908000C148C1408002100B40188
:10309000B501B201B3010800F112580B6D2892136B
:1030A0002800950122006D082800960008302000B5
:1030B00058020318701A6128580828001602073EA3
:1030C000960022000C108C10F01869283D00910128
:1030D0006B283D009001F115A32802305806031D0E
:1030E0009628A62098310330F11128009704950105
:1030F00022004C08280096002000640C0339013A95
:10310000031D862828001608F83E9600701E8C289D
:103110002100630828009600F018902800309128BC
:103120000130AB20983120001110A328033058063D
:10313000031DA32828001708FC39023897009501C1
:103140002100D801F1162100D80A08009D180800B6
:103150009D1470130800F5007508031DB128C626DC
:103160009831750B0800CD2608002000491808008A
:103170005E080339023A0319832AF01CC3285E084B
:1031800003390319CA28F018B5295E080339013A32
:10319000031DB52922000E1C202920005215D2182B
:1031A000F3283D0087269831031DDB2822008E1C62
:1031B000DB28812698316F269831031DE4282200F0
:1031C0000E1DE42875269831F2269831031DEC284F
:1031D00022008E1DEC287B26E0303D0092058A31CE
:1031E000AA229831F928ED2698310319F9280123EC
:1031F0009831ED269831031D20292000D21C20296A
:1032000022000E102000620E0339023A031D0A2923
:1032100022008E106F269831031D102922000E11F6
:1032200020005E0E0F39093A031D182922008E1165
:103230000A2698312C269831611E202901279831C1
:1032400022000E1C0C19AB29210026082704031D9F
:10325000AB293D0099269831031D362922008E188E
:1032600036292000491F3629812698316326983156
:10327000031D422922000E19422920004B1C42291D
:1032800075269831F7269831031D4E2922008E1994
:103290004E292000CA1E4E297B26983101239831E1
:1032A000FC269831031DA1292000D218A129210054
:1032B00050085104031DA129BF269831031D672919
:1032C000491F652922008E14672922008E1063266B
:1032D0009831031D72294B1C702922000E1572298A
:1032E00022000E11F7269831031D7D29CA1E7B2965
:1032F00022008E157D2922008E11E82598312000AC
:10330000903052115926983103197E2AA2269831FD
:10331000031D8F29F4302100D0000130D10020009E
:10332000611E08002C3059269831031D9929083058
:10333000132F4C0E890C0339023A031D0800643028
:10334000132F210050085104031908000130D00246
:103350000030D13B0800210026082704031908008B
:103360000130A6020030A73B0800F018BB295E0818
:1033700003390319C229F01C08005E080339013A19
:10338000031D080022000C1D142A20005215D2181B
:10339000EB293D0099269831031DD32922008E1C6C
:1033A000D3298126983163269831031DDC29220018
:1033B0000E1DDC2975269831F7269831031DE42966
:1033C00022008E1DE4297B26E0303D00A0058A31D5
:1033D000AA229831F129FC2698310319F1290123F9
:1033E0009831FC269831031D142A2000D21C142A7F
:1033F000B3269831031DFE2922008E1063269831D2
:10340000031D042A22000E1120005E0E0F390A3A15
:10341000031D0C2A22008E11E82598312C269831A4
:10342000611E142A0127983122000C1D0E18AB29A9
:10343000210026082704031DAB293D00872698316B
:10344000031D2A2A22008E182A2A2000491F2A2A10
:10345000812698316F269831031D362A22000E19D5
:10346000362A20004B1C362A75269831F2269831D0
:10347000031D422A22008E19422A2000CA1E422A17
:103480007B26983101239831ED269831031DA1291F
:103490002000D218A129210050085104031DA129A0
:1034A00022000E142000620E0339023A031D5F2A27
:1034B000491F5D2A22008E145F2A22008E106F267B
:1034C0009831031D6A2A4B1C682A22000E156A2AAD
:1034D00022000E11F2269831031D752ACA1E732A86
:1034E00022008E15752A22008E110A26983120009E
:1034F0009030521159269831031D86290A30210037
:10350000D000D1018F29541CBE2AF0189E2A5215D2
:10351000B3269831031D932A5F1E912A22008E1430
:10352000932A22008E1063269831031D992A2200C7
:103530000E1122000E14200052110800F01C080089
:1035400052155E19A62A22000E10B92A620E0339FE
:10355000023A031DB32A5F1EB02A22008E14B92A34
:1035600022008E10B92AAE269831031DB92A2200F6
:103570000E1122000C15200052110800F018DC2A50
:103580005215BF269831031DCC2A5F1ECA2A22007D
:103590008E14CC2A22008E1063269831031DD72A60
:1035A0005F1ED52A22000E15D72A22000E112200F6
:1035B0000E10200052110800F01C080052155E1970
:1035C000E42A22000E14FC2A620E0339023A031D7B
:1035D000F12A5F1EEE2A22008E14FC2A22008E1091
:1035E000FC2AAE269831031DFC2A5F1EFA2A22000F
:1035F0000E15FC2A22000E1122000C11200052117F
:1036000008002000D21C080021003708031D422BAF
:10361000A0302500160203180F2B960A152BA03098
:103620001606031D152B2000D21021005F08F83E5E
:10363000B7008F31322798310319541C282B2100F1
:1036400037082000A7000530BB2598312100B700BE
:1036500069269831031D2F2B2100B7363E2BA22659
:103660009831031D3E2B210037082000AA00AA36FE
:10367000AA36AA362A0821003702B7002000611EA8
:103680000800062FB7030800200052190D2C590816
:103690005806031D5E2B59085B020318532B59086B
:1036A0000319532BD9035B085902031CF01B592B38
:1036B000D90A5908532698312100C9002100490828
:1036C00074060319792B560857040319F119792B3D
:1036D0009631D4269831D4268A31F8229831F400D4
:1036E0007408031D792B8E31B3269831D22498317A
:1036F000F213740821004906031DF02B200051111C
:103700005908D8001A305802031C902BBA26983159
:10371000B735B80DA72698310318B80ABF30C52BA6
:1037200014305802031CAA2B5808A731D32798310C
:10373000A331D923983128082200B8002000270897
:103740002200B700210063082200B7070318B80A57
:10375000D830C52B0F305802031CB62BBA2698312F
:10376000A72698310318B80AEB30C52B0830580249
:10377000031CC92B58082200B700B80121006308B8
:103780002200B7070318B80AF930B707031CB803BB
:10379000CE2B210063082200B700B80101303802A7
:1037A000003003193702031CD82BFF30B700B801D3
:1037B0003708CC00163020005802031CE42B2100EF
:1037C00060082200CE00E62B2200CE01200058081F
:1037D0002200EF00EF36EF36EF366F08033CCD00E6
:1037E0002000580853269831740603190D2C5908E7
:1037F00058020318FD2B521B022C58085902031CB7
:10380000D21E0D2C5808D900532698312100C9002A
:10381000200059354A269831AB007408031D232C2B
:1038200020005808031D232CF11E182C2100921093
:103830002200E301E401F1118E31B3269831F01535
:10384000D2249831F21305307402031C2B2C210072
:10385000141A2B2C141605307402031C3F2C210063
:1038600092183F2C200060080F39063A03193F2CAC
:103870005F080F39063A03193F2C210092140530D6
:103880007402031CF11E462C210092100F27983160
:1038900003193506031D522C4808031D522C200025
:1038A000CB1E5F2C2100320F582C330A03195F2CDA
:1038B0002200470A1E3003194806031D612C7215A9
:1038C000622C7211FF3021003302003003193202E2
:1038D000031C6F2C2000D9012100D601D701A8308C
:1038E0003406023003193506031D8C2C48080319D1
:1038F0008C2C2000CB1A8C2CCB1662080F3922009E
:10390000EF0005306F02031C8C2C2500B031A02085
:1039100098318631DD269831701A972CDC24983145
:103920000630740203189D2CD22498319D2C21005E
:1039300092189D2C9731A0279831701DBF2C230021
:10394000210874020318A72C2000E7269831740878
:10395000031DBF2C20005A08031DBF2C5808031D4F
:10396000BF2CF111F0159631D42698312000521950
:10397000BF2CC72598317011F01FBF2CF013F01C1D
:10398000C32C0130C42C00302200EF00701CCA2C64
:103990000130CB2C00306F06031D08002000521DA3
:1039A000701108002100CC012200CF012100B801D4
:1039B0002000DA01E7260800200058085902031CFD
:1039C000E32C5835EE2C580859020318F12C5808EE
:1039D0005326983174020318F12C59354A26983130
:1039E000AB00053074020318FB2C2100AA01AB01C7
:1039F0002000CF01D00122005F086004031D3B2D91
:103A000021002B0820005002031D082D0A279831A1
:103A1000031CF01B3B2D70193B2DCF0A0319D00A54
:103A2000FE30A7004C0E890C0339BB259831AB0042
:103A3000FC30DB269831AC00003003180130AD00BB
:103A40002D0DAD0CAC0C2D0DAD0CAC0C2C08BB250C
:103A50002B07AE00210062082000AE020530A7004F
:103A600058089631DE2698312E021A3EB100220007
:103A7000DF00E001AD2D22005D085E04031DAD2DC9
:103A80002000500821002B02031D482DFB279831F0
:103A90000318AD2D01302000CF020030D03BF01FC5
:103AA000822D15305802031C572DB1015F2D2200C5
:103AB0004E082100600222004D072000B1002100C5
:103AC0002A0820004F0290269831153003192B0246
:103AD000031C722D16305802031C722DEC30CF07D8
:103AE000FF30D03D21002A0820004F029026983157
:103AF000213003192B02031CA92DF830CF07FF300A
:103B0000D03DA92D0930A70058089631DE269831FE
:103B1000AB004C0E890C0339AC00FE30DB2698312B
:103B2000AD00003003180130AE002E0DAE0CAD0C10
:103B30002E0DAE0CAD0C2D08BB259831AF002C0816
:103B40002F02B0002B08300221006107073E200041
:103B5000B10031082200DD00DE011E3020005802D5
:103B6000031C080021002B082000D00021002A0897
:103B70002000CF000800A900A80127082918A807DD
:103B8000A735A9362908031DBD2D28080800F119FD
:103B900008007018DA2DC626983121008E162300F1
:103BA0008E1621001D08033954389D000E12220084
:103BB0000E12F010701C0800CD269831E1261D0869
:103BC000033950389D008E1222008E12F014080026
:103BD00022000E10E0303D0092052000620E0339F5
:103BE000033A031DF62DE0303D00A1052000600ED4
:103BF000890C0339033A031D002EE0303D00A20575
:103C000020005E0E0F390A3A031D0800E0303D0027
:103C1000A305080022000C11E0303D00A0052000A3
:103C2000620E0339023A031D182EE0303D00A10553
:103C30002000600E890C0339023A031D222EE03069
:103C40003D00A20520005E0E0F39093A031D080051
:103C5000E0303D00A305080080302100A6000C30B4
:103C6000A70020004C0E890C0339033A031D3D2E9A
:103C7000F4302100A6000130472E4C0E890C033988
:103C8000023A031D482EF0302100A6000A30A7009A
:103C900020000800A03E860002308700403F21003F
:103CA000AA00413F0800A03E8600013087000108BD
:103CB00008002100D0000130D10020004C0E890CFA
:103CC0000339033A08002000600E890C0339033AD7
:103CD000080020004C0E890C0339033A080020002C
:103CE000600E890C0339023A08003D002208E039D1
:103CF0000D38A20008003D002308E0390D38A3006C
:103D000008003D002108E0390D38A1000800200816
:103D1000E0390D38A0002000620E0339023A080095
:103D2000AB0021002B082000503BAC0000302C02DF
:103D300008001208E0390D3892002000620E0339A5
:103D4000033A08004C0E890C0339023A0800B735D3
:103D5000B80D210063082200B7070800600E890C27
:103D60000339023A080022000C112000620E0339C8
:103D7000033A080058082200B700B80108002200E2
:103D80000C152000620E0339033A080022000C14BF
:103D90003D00900102309100080022008C143D008B
:103DA0009101023090000800200051157408C700EE
:103DB000210049080800A7004C0E890C0339013E78
:103DC000080021000E1623000E1621000800CF0166
:103DD000D0012100AA01AB0108003D0020081F39D5
:103DE0000D3A080020005E0E0F39093A0800200045
:103DF0005E0E0F390A3A08003D0012081F390D3ACD
:103E00000800C8302100A600A70108002100B70162
:103E1000B70A080021002A0820004F020800D0300D
:103E20002100340602342100D000D1010800200016
:103E3000B4000130B7012300EA020030EB3B6A080E
:103E40006B04031D522FEA01EA0AEB0121009D1CBD
:103E5000701B3A2F552798312F08B6002E08B50051
:103E60003608B3003508B200B336B20CB336B20C24
:103E70003208B7002000511C502F51109631D42623
:103E800098312100D601D701200034082100C90053
:103E9000FF302300EA002F30EB0022000E14522FD7
:103EA00022000E102000370808002000B001B101E8
:103EB0002200CB0A8927983122004B086C06031D8B
:103EC000832F200051142300DB01DC0122004A086B
:103ED0002000A700A80123005E082000AA002300FC
:103EE0005D082000A9008D313E2598312808B100D9
:103EF0002708B00031082200B60020003008220058
:103F0000B5009631D42620003108AF003008AE004D
:103F1000080021001C082200DC00DB0121001B0836
:103F20002200DB070318DC0A7017200051199D2FAF
:103F30002300213674020318A42F200051112300FE
:103F4000DD01DE012200CA0122005C08B6005B0828
:103F5000B5005B082300DD0722005C082300DE3D7E
:103F60002200CA0A701A080035083604031DBA2F49
:103F7000F214BB2FF2102000500822003602031D5D
:103F8000C52F20004F08220035020318DB2F230025
:103F900021087402031CD82F2000500821002B0296
:103FA000031DD42FFB279831031CD82F2000D117D5
:103FB00020005210E82F360820005002031DE42F85
:103FC0002200350820004F020318E82FD1135214A5
:103FD0002300210874020318EF2FF01BF72F21088C
:103FE00074020318080020005B08031D080020006D
:103FF000D1135214080020004F0821002A020800A3
:10400000FF3FFF3FFF3FFF3FFF3FFF3FFF3FFF3FC0
:10401000FF3FFF3FFF3FFF3FFF3FFF3FFF3FFF3FB0
:10402000FF3FFF3FFF3FFF3FFF3FFF3FFF3FFF3FA0
:10403000003480343F3402340034013400340A3414
:10404000003418340034CD34043402340034703475
:1040500000340C3400347B340034043401343D34F7
:104060005534C83400341634003425340034023456
:1040700000340134063408340B340A340634043472
:104080001E340134043408341A3405340134033442
:1040900001340C343E34013401341E344034FF34D6
:1040A0000234E327A031031DAD28F627A031031DFC
:1040B0005E2861080339013A03199E28F627A031CA
:1040C000031D912861080339023A031D7A287408F8
:1040D000031D6F282100300831040319E82820004F
:1040E0005B080319BE294B18842822000E11A8274B
:1040F000A031BE2961080339033A031DBE295B08BC
:10410000031987284B1D752822000E15772874087F
:10411000031DBE29210030083104031DBE292000E3
:10412000AA2861080339013A031DBE299E31AE2633
:10413000A031031DA128F01C5219BE294B18EB28F1
:10414000EE28600E890C0339033A0319F01CBE29CE
:104150005219BE294B1CEE28EB2860080F39023A91
:10416000031DF128CB1CB6280130B7280030AD0064
:104170004B1CBC280130BD2800302D060319E32854
:104180004B0C890C0139013CAD00AD0DAD0D220089
:104190000E0820002D06FB392D0622008E0021007E
:1041A0006F082000A7003130A801A900AA01D92377
:1041B000A03128082200EA00200027082200E90098
:1041C00020009E27A031220069086A04031DBE2931
:1041D00020004B1DEE2822000E15BE2922000E11D4
:1041E000BE2960080F39033A03195F1A4D29CB1C09
:1041F000FB280130FC280030AD004B1C01290130A8
:10420000022900302D06031908294A149E27A031DF
:104210004A1C6F2926001208031D2A2922000E11AC
:10422000AE27A03121006D082600920021006C0805
:104230002200C500C60121006C082200C300F03036
:10424000C401C30EC40EC40543080F39C404F030C2
:10425000C305BE29220045084604031D382926004F
:10426000120821006D06031D38296D36CD006C291A
:104270000030220044022130031943020318BE29F2
:104280002600120821004D06031DBE292E082F040A
:10429000031D9C2920004A106F2960080F39043A39
:1042A000031DA229541C56295F1A58295F1A742924
:1042B0004B1C6F2922000E15AE27A03121004C089F
:1042C0002000AD00AD36AD36AD365A352D0774073A
:1042D0004C27A03169086B0726009200BE292600F2
:1042E000920122000E119E295F1A5418BE294B1804
:1042F000992922000E1121004C082000AD00043045
:10430000AD36890B80297408AE00AE365A352E07BB
:104310002D074C27A0316903FF3A2000AD00210092
:104320006B0820002D02A03E26009200AE27A0318F
:10433000BE29A0302600920022000E15E0303D007C
:10434000A205BE2960080F39053A031DB1294B08A3
:104350000139AD00AD0E4C082D06EF392D06CC000D
:10436000BE2960080F39063A031DBE29F11A4B1CFD
:10437000BC2921009210BE2921009214200060085F
:104380000F39013A0319C92960080F39043A031D8E
:1043900008006119711808007408031D08005F1EE9
:1043A000D4295F1A541CD92922000E11260092012B
:1043B00008005F1A5418080022000E15A0302600CD
:1043C0009200080043085002031DE82942084F02EA
:1043D000031C032AD1105008A8004F08A700420868
:1043E000A7024308A83B6430A900AA01D923A03141
:1043F000DE278631FE26A0312F08C5003008C60012
:104400003108C700072AD114C501C601C7014F08EA
:10441000500403192C2A5008B0004F08AF00863111
:10442000FE26A0312F08B3003008B4003108B500D3
:104430004508B6004608B7004708B8006B26A0310B
:1044400033082200A300200034082200A40020002A
:1044500035082200A5002E2AD927A03120004F08B8
:104460005004031D342AD92720004508C2004608FD
:10447000C3004708C4000800BA2796310B26A031B4
:10448000240044060319462AFF30562ABA279631DB
:104490000B26A03124004406031D5C2A50309631BF
:1044A0000B26A0315A3A03195C2A5A302000C70063
:1044B00050308631DD26A031B42796310B26A0314D
:1044C000240044060319662AFF30762AB427963161
:1044D0000B26A03124004406031D7C2A543096315B
:1044E0000B26A0315A3A03197C2A5A302000C70003
:1044F00054308631DD26A031643096310B26A03150
:10450000003A03198A2A643096310B26A031FF3A0B
:10451000031D902A9731DC27A0318631DD26A0319A
:104520004B3096310B26A031013A031D9C2A0130F5
:1045300090313520A0319E2AA122A031EE23803176
:104540005628503096310B26A0315A3A031D282B9D
:10455000523096310B26A0315A3A031D282B543085
:1045600096310B26A0315A3A031D282B553096312F
:104570000B26A031003A0319CA2A553096310B2672
:10458000A031EC27A0310318CA2A553096310B26EA
:10459000A031CB2A02302500A200A301023E220056
:1045A000EB000230FA001F307A020318C42B7A089D
:1045B000543E96310B26A03196319426A031C02767
:1045C00023005F082000C100230060082000C20013
:1045D000230061082000C30096311D26A0318731D9
:1045E0003827A03184318C24A0316827A0312608D7
:1045F000C03F2708C13F22006B082400B300B4016C
:104600007A35A03E7A27A031031C122B6827A031EF
:10461000403FB300413FB4007A359E3E7A27A03137
:10462000031C262B7A359E3E860002308700403FD1
:10463000B300413FB4003308023EB5000030343DC2
:10464000B6007A35A03E8600F127A031FA0AD32AB7
:10465000FA012030FA0A7A020318B12B7A03031DFB
:104660005A2B553096310B26A031003A0319452BB1
:10467000553096310B26A031EC27A0310318452B7D
:10468000553096310B26A031552B04302500A20061
:10469000A301FB27A031031D4F2B0330552B5608D8
:1046A0000339033A0230031D592B2500A2000230C2
:1046B000A301FA00FB27A031031D7C2B0230A03E92
:1046C0008600023087007A08D327A031D923A03191
:1046D000403F27072400B300413F2000283D24002D
:1046E000B4003308FD3EB500FF30343DB600682706
:1046F000A031F127A0319B2BA23086000230870029
:104700007A082400B300B401B335B40DB335B40D49
:10471000403F3307B500413F343DB6003508FC3E0D
:10472000B700FF30363DB8007A35A03E8600370826
:10473000C03F3808C13F8731D627A031031D292B40
:104740006827A031403F2400B300413FB400B43695
:10475000B30C7A35A03E86003308C03F3408C13F11
:10476000292B523096310B26A0315A3A0319C42B0B
:10477000B0319320A0318631DD26A0319731F32767
:10478000A0318631DD26A03125000030A001A10135
:104790005D02E83003195C020318D52B5C08183E53
:1047A000DE0000305D3DDF000800FF30DE00DF018D
:1047B0000800AB01AC01271CE12B2908AB072A0834
:1047C000AC3DA935AA0DA836A70C27082804031D5F
:1047D000DB2B2C08A8002B08A70008002300A00151
:1047E000701A212C533096310B26A0312300A100E2
:1047F0000230FA0020307A020318212C7A08A03EF9
:104800008600013087007A08453E8400023085002A
:1048100000082000AB007A089F3E8400013085002C
:1048200000082B0781007A08A03E8600C3300102F1
:10483000031C1F2C7A08A03E8600C2308100FA0AB1
:10484000FA2B701E732C2000D21D732C56080339CE
:10485000023A03194D2CFA011730FA0A7A020318AA
:104860003A2C7A08A03E8600013087007A08043E80
:1048700081002C2C1C302300B7001E30B8002130E2
:10488000B9001A30FA0020307A020318732C7A0823
:10489000A03E8627A031FA0A432C56080339023A73
:1048A000031D732CFA011530FA0A7A020318612CE1
:1048B0007A08A03E8600013087007A08083E810011
:1048C000532C21302300B5001630FA0020307A0234
:1048D0000318732C7A08A03E8627A0312030FA0AEC
:1048E0007A02031C6A2C21002030BA01B901FA00B7
:1048F0007A0803190800A03E8600013087000330C3
:104900002000A70023003F089631DE26A0310102D7
:104910007A08031C8E2C2100BA007A08A03E86007B
:104920000130870023003F082000AB00AB36AB36D8
:104930002B080102031C9F2C7A082100B900FA03FE
:10494000782CB4302200C90023082000C1002200C6
:1049500024082000C200220025082000C300B43033
:1049600096319426A031C02796311D26A0314108EA
:104970002200A000200042082200A10020004308DD
:104980002200A200230021087402031CF62C22003E
:1049900020082000B600220021082000B7002200D5
:1049A00022082000B800CD27A0316B26A031922725
:1049B00084318C24A03126082200CF00053020004D
:1049C0005802031CEB2C2100650A2200E82CCF368C
:1049D000890BE72CF62C210066082000A700220096
:1049E0004F089631DE26A0312200CF002000D11CD6
:1049F0001F2D220022082104200403191E2D20004F
:104A00008030BB01BC003F30BD00220020082000E8
:104A1000BE00220021082000BF0022002208200042
:104A2000C000843171243B082200A00020003C0813
:104A30002200A10020003D082200A200CF01220098
:104A40004F082100B8000800210049080319522E20
:104A50002000D11F1E2E210038082400B300B4010D
:104A6000B309B409B30A0319B40A3408B6007408C8
:104A70003302B500031CB603C23EB7000030363D1A
:104A8000B800803AB90080303902031D4B2D200058
:104A90005A0824003702031C1E2E740803191E2E08
:104AA00006302000AF00B0014C0E890C0339240001
:104AB000B300B401B335B40D33082000AF022400B5
:104AC00034082000B03BAF35B00DAF35B00DC72670
:104AD000A0312F08B3003008B4003108B50022001F
:104AE00023082000B600220024082000B70022007E
:104AF00025082000B8006B26A03133082200D6001C
:104B0000200034082200D700200035082200D800F9
:104B100059085A04031D142E2000DA0AC727A031B1
:104B2000200058082200D9070318DA0AFB30D907F9
:104B3000031CDA03740823002402031CA92D740843
:104B400021004902031CA92D20005212C727A031C1
:104B5000AB2D200052162000B401B501B601220091
:104B600056082000B700220057082000B800220095
:104B700058082000B9002027A031031C521E092E1E
:104B800022005A082000A800220059082000A7008F
:104B90006430A900AA01D923A031DE278631FE2680
:104BA000A0312F082300C000200030082300C100DE
:104BB000200031082300C200220056082000B30064
:104BC000220057082000B400220058082000B50039
:104BD00023006E27A0316B26A03133082300C000CC
:104BE000200034082300C100200035082300C20043
:104BF0006E27A031CD27A0316B26A03192278431BA
:104C00008C24A03127082200DA0024002608220084
:104C1000D900200058085B020318182E2200D9354D
:104C2000DA0DD935DA0D182E0130D9020030DA3B11
:104C30002000D1132300E801E80AE9012000521CFA
:104C4000522E5A080319522E521023006808690484
:104C5000031D4E2E093020005A020318472E04303F
:104C60002300E8000730E9012000A700580896312A
:104C7000DE26A0312400B3002300E802031CE90370
:104C8000E835E90DE835E90DE80A0319E90A2100DC
:104C90003808031DB8032000DA03522E0130E80261
:104CA0000030E93B740820005A072400B300B40127
:104CB000B40D3408803A803C031D612E3308230074
:104CC00021020318080023002108740203180800B9
:104CD0002000DA0108003608B9003708BA003808A1
:104CE000BB0003103A0D3B0DC0004008031D792E98
:104CF000E82F3308B9003408BA003508BB000310A8
:104D00003A0D3B0DC1004108031D872EE82F893065
:104D1000BD01BE01BF014107B900C0023808C10092
:104D20003508C1068030C1051830B717B801B4176F
:104D3000B501BC00BD35BE0DBF0D35083802031DE1
:104D4000A72E34083702031DA72E33083602031C92
:104D5000B02E3308B6023408B73B3508B83B3D14D3
:104D6000B635B70DB80DBC0B9A2E3D08A7003E080E
:104D7000A8003F08A9004008AA004108AB00E226AD
:104D80002708B3002808B4002908B5000800B201BC
:104D9000B01FD12EAF09B009AF0A0319B00AB20192
:104DA000B20A2F08A7003008A8008E30A901AA0077
:104DB0003208AB00E2262708AF002808B000290817
:104DC000B10008002A080319EA2E2908280427043C
:104DD000031DF22EA701A801A9010800AA0AA936FD
:104DE000A80CA70CFE3029050319002FEE2EAA0AE5
:104DF000A70A0319A80A0319A90AA936A80CA70C1F
:104E0000FF30290503190D2FF72E02302A02031C4B
:104E10000F2FAA03A735A80DA90DA81F052F2A1C1F
:104E2000A813AA362A08AE00AD01AC012C08A704CD
:104E30002D08A8042E08A9042B08031DA917080093
:104E4000B61F2F2F3408003CB4003508031C350F63
:104E5000003CB5003608031C360F803CB600B91F75
:104E60003E2F3708003CB7003808031C380F003CC1
:104E7000B8003908031C390F803CB9008030B606F1
:104E8000B90639083602031D080038083502031D2B
:104E900008003708340208002100EB006A080A3EC7
:104EA0002000AD00003003180130AE00803AAF00A2
:104EB00080302F02031D602F21006B0820002D027F
:104EC0000318662F21006A080A3EEB002100080043
:104ED0007A35A03E86000230870008004008200096
:104EE000B600230041082000B7002300420820003C
:104EF000B80008008600403FB500413FB6003408C6
:104F00003602031D08003308350208008600013010
:104F100087007A089F3E8400013085000008043E27
:104F20008100080033082400A60020003408240073
:104F3000A700200035082400A80008004B0801390C
:104F4000AD00AD0D4B082D06FD392D06CB00080038
:104F50007E302100B0000230B10008003D00220880
:104F6000E0390E38A200080020005508033924005B
:104F7000C40073342000560803392400C40051349F
:104F80002F08C4003008C5003108C6000800210001
:104F900064082200D900DA010800C830B301B40067
:104FA0004230B5000800A7000330A801A900AA01FB
:104FB00008002200A301A401A50108002808B000F0
:104FC0002708AF000800200060080F39013A0800E8
:104FD000B301B401B50108002400B3001530330259
:104FE00008003508C03F3608C13F0800600E890C34
:104FF0000339013A0800200056080339023A080034
:10500000FF3FFF3FFF3FFF3FFF3FFF3FFF3FFF3FB0
:10501000FF3FFF3FFF3FFF3FFF3FFF3FFF3FFF3FA0
:10502000FF3FFF3FFF3FFF3FE51C44282930570269
:1050300003182A2857082100E60066082000C70048
:1050400020308631DD26A8315A302000C7001F30BD
:10505000AA31402A29305702031CC0288130570248
:10506000031C34288030D7005708D83E2100E500C3
:1050700065082000C7001E308631DD26A8315A3071
:105080002000C7001D302828651D5B280530570209
:1050900003184C280530D70057082100E4002000F1
:1050A0005708C70022308631DD26A8315A3020004B
:1050B000C70021302828E51D72280A30570203183E
:1050C00063280A30D70057082100E3002000570862
:1050D000C70024308631DD26A8315A302000C700B1
:1050E00023302828651E93280730570203187A2892
:1050F0000730D70051305702031C80285030D700AA
:10510000570857075707013ED7002200ED0020003F
:105110005708C70026308631DD26A8315A302000D6
:10512000C70025302828E51EC2283D305702031C41
:105130009B283C30D700570896319426A831BB31C4
:10514000DE23A831E100B931A321A831BB31C52349
:10515000A83196311D26A831BB31D223A8312000B9
:105160005708C70028308631DD26A8315A30200084
:10517000C70027308631DD26A831A231A122A8310F
:10518000AA31432A651F1E290B3057020318CC2869
:1051900057082100E200E528153057020318D928E6
:1051A0000B305702031CD9285708F63E2100E100B6
:1051B000E528333057020318E52815305702031C41
:1051C000E5285708EC3E2100E0002A3096310B26F6
:1051D000A831210062060319F42862082000C700E4
:1051E0002A308631DD26A8312B3096310B26A831A6
:1051F000210061060319032961082000C7002B3034
:105200008631DD26A8312C3096310B26A8312100BD
:1052100060060319122960082000C7002C3086316F
:10522000DD26A831293096310B26A8315A3A0319C8
:10523000C0285A302000C70029302828B331ED2B70
:10524000681C40290430D70757082300A10020001C
:105250005708C70053308631DD26A931B03193207D
:10526000A9318631DD26A93102302500A200A30133
:105270002000C70055308631DD26A931BC31D62C3F
:10528000E81E681B4529E81F8629213057021F3078
:105290000318D700D70521006708031952294808C9
:1052A0002000DB002000E81E642957082100C5000B
:1052B00020005708C700AB308631DD26A9315A30AF
:1052C0002000C700AA30402A681F7529570821000E
:1052D000C40020005708C700AD308631DD26A93153
:1052E0005A302000C700AC30402AE81F432A570834
:1052F0002100C30020005708C700AF308631DD26EB
:10530000A9315A302000C700AE30402A661EA229BB
:10531000083057020830031CD70080305702031CA6
:1053200093297F30D70057352100EC006C0820000E
:10533000C70030308631DD26A9315A302000C70041
:105340002F30402AE61EE42905305702031CAA2903
:105350000430D70057082100ED0020005708C7008F
:105360002E308631DD26A9315A302000C7002D307D
:105370008631DD26A9312E3096310B26A931013A2E
:10538000031DC4292830DE292E3096310B26A93181
:10539000023A031DCD295030DE292E3096310B26DE
:1053A000A931033A031DD6298030DE292E309631EB
:1053B0000B26A931043A031DE029A0302100ED009D
:1053C000B7318C27A931432A661FFB297B3057024E
:1053D000031CEC297A30D70057352100E900690811
:1053E0002000C70032308631DD26A9315A30200036
:1053F000C7003130402A671F0C2A57082100EF00F0
:105400006F082000C70034308631DD26A9315A30BC
:105410002000C7003330402AE71F1D2A570821000B
:10542000DD0020005708C70036308631DD26A9315F
:105430005A302000C7003530402A681D2F2A5708EF
:10544000E73C2100DC005C082000C70016308631F4
:10545000DD26A9315A302000C7001530402AE81C4B
:10546000432A5708E73C2100DB005B082000C70007
:1054700018308631DD26A9315A302000C700173098
:105480008631DD26A931B931DA21A9316712E71257
:105490006711E711B0314620A931B0318720A93119
:1054A000B0316A20A9314C124C11CC10C9104911ED
:1054B00049104A1121009214592F2000D4145D087C
:1054C0002100C70020005C082100C6005E2FBA3111
:1054D0001B22A931B936890B6A2A02303906031D0D
:1054E0000D2B2000630C890CB931D221A931073072
:1054F000BA36890B782A3A08B0312620A9314A08F1
:10550000B0318120A931CA00630CB931EE21A93133
:1055100020005C082400BB000630BB36890B8D2AB6
:105520003B0801393A06BC00BC0EBC0DBC0D200086
:105530004A0824003C06BF393C06B0317B20A93123
:105540000630B936890BA12A39080139BA00BA0CDC
:10555000BA0C20004A0824003A067F393A06B031D6
:105560007B20A9310430B936890BB32A01303905C3
:10557000BA002000600E013924003A06BB0020006A
:105580004B0824003B06FE393B062000CB004B11A4
:105590005F1A5418CE2A01304B15CB066308B93177
:1055A000D221A9310530BA36890BD32A3A080139FC
:1055B000B0312620A9314B08B0318120A931CB0070
:1055C000B931E821A93139080339BA00BA0EBA0D48
:1055D00020004C0824003A069F393A062000CC00EF
:1055E000B0318D20A93120004D0C890C03392400E5
:1055F00039060319FE2A2100D736D60C2000B03117
:105600008D20A931B90DB90D20004D0824003906AF
:10561000F33939062000CD005E2FBA311B22A931A3
:10562000B936890B102B03303906031D5E2F20007D
:10563000D41C5D2AB031B120A931031D5D2AB931D6
:10564000E821A931BA311222A931031D5D2A2000B7
:10565000D410DC1B1C2D0330B931C621A931033A0B
:10566000031DB92BB931F521A931031D3A2BCF30D8
:10567000E3057C2BB0314120A931390B432B973105
:10568000E527A9314D2BB9319D21A931023A031DDE
:105690004F2B20006308CF392038E3007C2BB93131
:1056A0009D21A931033A031D592B30302000E3041A
:1056B0007C2BB9319D21A931043A031D622B2000B6
:1056C00063137C2BB9319D21A931053A031D6B2B46
:1056D000200063177C2BB9319D21A931063A031DA7
:1056E000742B2000E4177C2BB9319D21A931073A96
:1056F000031D7C2B200065142000630E0339240059
:10570000B900043096310B26A9312400390603195B
:10571000982B2000630E0339C70004308631DD2644
:10572000A9315A302000C70003308631DD26A93167
:105730002000630EB0315E20A931063096310B2671
:10574000A931240039060319B52B00302000631B52
:105750000130C70006308631DD26A9315A302000DD
:10576000C70005308631DD26A93180315620A931A8
:10577000A62C0330B931B121A931031D0C2CB9314C
:10578000F521A931031DC62BE714A62C07305C05B3
:105790002400B9003903031DD62B20007F30671485
:1057A00096310B26A9312200D300A62CB9319D21B8
:1057B000A931023A031DDF2B2000E617A62CB931D0
:1057C0009D21A931033A031DE82B20006815A62C62
:1057D000B9319D21A931043A031DF12B2000E814B1
:1057E000A62CB9319D21A931053A031DFA2B2000C1
:1057F000E816A62CB9319D21A931063A031D032CC8
:1058000020006817A62CB9319D21A931073A031D44
:10581000A62C2000E817A62CB931CC21A931390BD0
:10582000542C20000730B931C621A931053A031D97
:105830001C2C2000E811362CB9319D21A931063AE3
:10584000031D252C2000E815362CB9319D21A931E6
:10585000073A031D362C20001B30E415C701C70A88
:105860008631DD26A9318431E124A9312000680C7C
:10587000B931EE21A9310C3096310B26A931240023
:105880003A060319A62C00302000E8190130C700A1
:105890000C308631DD26A9315A302000C7000B308C
:1058A0008631DD26A931A62C20005C080339031DB2
:1058B000A62CB0311B20A931031D692C1C306417A4
:1058C000C701C70A8631DD26A9318431E124A93117
:1058D000A62CB0314120A931390B712C2000E514E0
:1058E000A62CB9319D21A931023A031D7A2C200042
:1058F0006515A62CB9319D21A931033A031D832CCE
:105900002000E515A62CB9319D21A931043A031DCB
:105910008C2C20006516A62CB9319D21A931053AA1
:10592000031D952C2000E516A62CB9319D21A93127
:10593000063A031D9E2C20006517A62CB9319D2127
:10594000A931073A031DA62C2000E51721004208C3
:10595000031D112D2000660D660D01392400B900CC
:105960002000650CB0310720A931650CB031012051
:10597000A931650C01392400BD002000640E890C9A
:10598000890C01392400BE0020006508013924007B
:10599000BF002000640D640D013924003F073E075D
:1059A000B0312D20A9312000670C01392400B90045
:1059B0002000650D650D01392400BA002000650E38
:1059C000890CB0310F20A931650EB0310120A93109
:1059D000650E01392400BD0020006708013924004C
:1059E0003D073C07B0312020A9312000680D680D2B
:1059F00001392400B9002000680EB0313A20A931E5
:105A0000680EB0310F20A931680C01392400BC00A8
:105A10002000680C890C013924003C07B03120209B
:105A2000A93102304202031C592FB931DA21A931C0
:105A3000B0316A20A931572FC0305C052400B9006D
:105A4000803A031D122E20000330B931C621A9313E
:105A5000033A031D4C2DB931F521A931031D322D17
:105A60006716CF2DB0314120A931390B3A2D2000D6
:105A7000E716CF2DB9319D21A931023A031D432DDF
:105A800020006715CF2DB9319D21A931033A031D9F
:105A9000CF2D2000E715CF2D0330B931B121A93129
:105AA000031D732DB931F521A931031D592DE616BA
:105AB000CF2DB0314120A931390B612D2000661660
:105AC000CF2DB9319D21A931023A031D6A2D200045
:105AD0006617CF2DB9319D21A931033A031DCF2D72
:105AE00020006717CF2DB931CC21A931390B7F2D7B
:105AF000B931F521A931031DCF2DE717CF2D200096
:105B00005C080339031DCF2DB0311B20A931031DC3
:105B10008B2D5F12B22DB0314120A931390BA12D4F
:105B200020005F166008F0390138E000B130C7018D
:105B3000C70A8631DD26A93122008E1420004917BC
:105B4000B22DB9319D21A931033A031DB22D200098
:105B50003B306416C701C70A8631DD26A93184317E
:105B6000E124A93120005F0E01392400B90038304A
:105B700096310B26A931240039060319CF2D0030A8
:105B800020005F1A0130C70038308631DD26A93188
:105B90005A302000C70037308631DD26A931210078
:105BA0004208031D052E2000670CB931EE21A931F2
:105BB0002000670CB0310F20A931670EB0310120F1
:105BC000A931670E013924003C073B073A07210041
:105BD000C2002000670EB0315E20A9312000660EA1
:105BE000B0313A20A931660E01392400BB002000F3
:105BF000660E890C01392400B0312020A931200023
:105C0000670D670D01392100C20702304202031CF3
:105C1000592F20006712E7126711E711B031872072
:105C2000A931572FC03020005C052400B900C03ACC
:105C3000031D592F20000330B931C621A931033A81
:105C4000031D672E20000730B931C621A931043A5F
:105C5000031D2D2E200066144D2EB9319D21A93132
:105C6000053A031D372EFC302000DE054D2EB931DC
:105C70009D21A931063A031D422E20005E08FC3901
:105C800001384C2EB9319D21A931073A031D4D2E03
:105C900020005E08FC390238DE0020005E0803396F
:105CA0002400B9003F3096310B26A9312400390673
:105CB0000319322F20005E080339C7003F308631B8
:105CC000DD26A9315A302000C7003E302F2F033087
:105CD000B931B121A931031DB62E20000730B931E9
:105CE000C621A931043A031D782E2000E614982E0F
:105CF000B9319D21A931053A031D822EF9302000CA
:105D0000E405982EB9319D21A931063A031D8D2E47
:105D100020006408F9390238972EB9319D21A93144
:105D2000073A031D982E20006408F9390438E4006E
:105D30002000640C03392400B900433096310B264F
:105D4000A931240039060319322F2000B0319C20DC
:105D5000A9318631DD26A931B031AD20A931863196
:105D6000DD26A9319631A526A931322FB931CC21B2
:105D7000A931390BD82E20000730B931C621A931FD
:105D8000043A031DC62E20006615322FB9319D211D
:105D9000A931053A031DCF2E2000E615322FB93167
:105DA0009D21A931063A031D322F20006814322F9D
:105DB00020005C080339031D322F0730B931C6219A
:105DC000A931043A031DE72E2000DE111C2FB93142
:105DD0009D21A931053A031DF02E2000DE151C2F50
:105DE000B9319D21A931063A031D0B2F22003D0830
:105DF0003E04031D0B2FE130BD000230BE00083011
:105E00002000E1060030E1190130C7004B30863137
:105E1000DD26A9311C2FB9319D21A931073A031D77
:105E20001C2F20004C30E416C701C70A8631DD263E
:105E3000A9318431E124A93120005E0CB931EE2171
:105E4000A9314A3096310B26A93124003A060319AC
:105E5000322F00302000DE190130C7004A30863171
:105E6000DD26A93121004208031D4F2F20006808BC
:105E700001392400B9002000660CB0310720A93197
:105E8000660CB0310120A931660C01392400BD0037
:105E90002000660801392400B0312D20A9310230DC
:105EA0004202031C592F2000B0314620A9312100A5
:105EB000C20121000C150E142000D217A031512070
:105EC000A93120005F1A672FB2313A22A9318D31F2
:105ED0006325A9318E313826A93120005F1E862F17
:105EE0005E08B931AB21A9310318862FBA310C22D3
:105EF000A931B33096310B26A931013A0319862F07
:105F0000B031A420A9318631DD26A93172190800EB
:105F10002000541DCB1E0800A13096310B26A9315C
:105F20002400B9007006FE393906F000A33096311E
:105F30000B26A9312400B90020004B08B0315220B3
:105F4000A931CB00A43096310B26A931BA310522F4
:105F5000A9314908B0314C20A931C900A53096318A
:105F60000B26A931BA310522A9314A08B0314C209B
:105F7000A931CA00A63096310B26A931B0311520BF
:105F8000A9314C08B0317020A931CC00A73096312E
:105F90000B26A9312400B90020004908B031522055
:105FA000A931C90062080F392400B900053039024F
:105FB000031CE02FA83096310B26A9312500920052
:105FC000A93096310B26A931B0311520A9314A08E4
:105FD00024003906DF3939062000CA00F01CF22FF0
:105FE0000130F32F00302400B900701CF92F01306C
:105FF000FA2F0030390603190800B0316420080078
:10600000FF3F890C01392400BC0020000800240057
:10601000BA00BA0C3A0C0139BB0020000800890C08
:1060200001392400BB00200008002400B900B90E8B
:10603000B90D20000800DC36DC365C0807390800A2
:106040003B073A0739072100C20708003906BB00A1
:10605000BB0DBB0DBB0D200008003D073C073B07F7
:1060600039072100C2000800200055080339240028
:10607000B9007334890C890C01392400BA0020005E
:10608000080007305C052400B90008006610E6101F
:106090006611E6116810080024003906BF39390678
:1060A0002000080024003906FE39390620000800C7
:1060B00057082400B900B90E20000800890C890C8B
:1060C00001392400B900080070152000DB01D2124C
:1060D000521708006811E810E8126813E813080066
:1060E000240039069F393906200008005608033974
:1060F0002400B90051342000CA005C082400B90013
:10610000080024003B06F7393B0620000800661211
:10611000E61266136713E71308004C0E890C033967
:106120002400B90008005A302000C70052344C0E39
:10613000890C0339013A0800640C0339C700433461
:1061400012082000C700A8342000B330C701C70AD6
:1061500008005A302000C70040345A302000C700E1
:1061600042342100470820005D0608000C12731E0F
:10617000CC2822006E08F50021005A0AC028F53606
:10618000890BBF287518C62822000C16E13073123F
:10619000280092009101080022000C1221005A08E8
:1061A000031D0800F3111312200013122200D10165
:1061B000D2017218E32887302000D3055308F8393C
:1061C0000238D3000800E5200800062ABF1C8F29EA
:1061D00020005308073903198F292422B031093AC6
:1061E000031D052953080739033A031DFC287210C3
:1061F00021003F187214052953080739013A031D7D
:106200000529F11321003F18F11720002422B03195
:10621000031918292422B031093A031911299C21A4
:10622000B03120002422B031A900A9032A22B031C4
:106230002422B031031D322953080739A900A90AC5
:1062400053082906F8392906D30087394038D30086
:106250000739033A031D32292422B031A900A90AC3
:106260002A22B0312422B031083A031D4C295308A8
:106270000739023A0319F11F402921003E08482935
:1062800053080739043A0319721C4C2921003C08B1
:10629000CF00CF13E421B031200053080739053A6D
:1062A000031D8F29F11B8D2921003E083C06031D8B
:1062B00063293D083B06031D63291C22B031F310FE
:1062C000731171178D293C093E06031D6F293D0886
:1062D0003B06031D6F291C22B031F31460293E08D0
:1062E0003C06031D7C293322B031031D7C291C226E
:1062F000B031F310731561293C093E06031D88294E
:106300003322B031031D88291C22B031F3147A29BD
:10631000F310731171132000D4100522B031210045
:10632000BF1C0800200053080739031D080053084C
:10633000F8390138D300080021003F18AC29BC29E6
:106340002100BE0ABC292100BD0ABC292100BC0ACB
:10635000BC292100BB0ABC29200053080739013A97
:106360000319A029033A0319A329013A0319A629FD
:10637000073A0319A929BC292000530CA700A70C30
:10638000270C0F39A80002302802031C0800D4296A
:106390002100BE3508002100BD3508002100BC35B4
:1063A00008002100BB35080053080739013A0319DA
:1063B000C829033A0319CB29013A0319CE29073A10
:1063C0000319D129E329080041304F02031CEA29AF
:1063D0000330CF024F086E06031D08001E30F31570
:1063E0006E020318F8296E08090709070338F9290E
:1063F000FB302200EE0020001312280092019101D0
:10640000210013160730DA000800062AF0302100B8
:10641000BF05C0012000530887394838D300F83041
:10642000D3052100FF30BE01BD01BC01BB01F1134A
:1064300072102200EE0008003E082000DD0021005E
:106440003D082000DC000800530CA900A90C290C11
:106450000F390800A90DA90DA90D53082906873980
:106460002906D3000800FC303B062000A9002100CB
:106470003D06080062080F39013A0319442A6208F0
:106480000F39043A031D772A62080F39013A031DB8
:106490004C2ACB1DD72AD42A62080F39043A031D8F
:1064A000A72B220067086804031D5E2A2000CB1D6D
:1064B0005C2A22008E145E2A22008E1074080319B2
:1064C000711CA72BF01FA72B5508031DA72B00300D
:1064D00021002D028D3003192C020318A72B220056
:1064E0008E140C30E700E801D501D50AA72B62080D
:1064F0000F39023A031DDA2A4B1ECB1D812A403088
:10650000C906BE23B231620E0339013A031D8C2A3B
:10651000D523B2310319D22A620E0339013A031D81
:10652000BD2AE123B231031DAC2A5B080319A32A5B
:10653000491F9D2A22008E149F2A22008E10A73107
:10654000A827B231A72B7408031DA72B2100300800
:106550003104031DA72BD72AE723B231031DA72B34
:106560005B08031D9D2A7408031DA72B210030081A
:106570003104031DA72B2000D22AD523B231031DDD
:10658000A72B620E0339023A031DCA2AF01C5219C6
:10659000A72BD22A620E0339033A0319F01CA72B4A
:1065A0005219A72B491FD72A22008E14A72B22008D
:1065B0008E10A72B62080F39033A031D352B4B1E93
:1065C000CB1DE32ACA14BE23B231CA1C322B2500CC
:1065D0001208031D062B22008E10CF23B23121009A
:1065E0006D082500920021006C082200C100C20144
:1065F00021006C08AE00F030AF01AE0EAF0EAF055B
:106600002E080F39AF04F030AE05A72B2200410849
:106610004204031D162B2500120821006D06031DE0
:10662000162B6D36CD0025009200A72B00302100DF
:106630002F02213003192E020318A72B2500120860
:1066400021004D06031DA72B2E082F0403192B2B09
:1066500022008E14642B25009201DB23B23120002E
:10666000CA10A72B25009201622B62080F39053A48
:10667000031D3D2BCB196A2B622B62080F39063A9A
:10668000031D732B4B1ECB1D472B4030C906BE2369
:10669000B231D523B231031D502B491B6A2B622B1B
:1066A000E123B231031D592B7408031D491F622BCE
:1066B000682BE723B231031DA72B5B08031D622B58
:1066C000491B682B22008E10E0303D00A105A72B4E
:1066D000491FA72BA83096310B26B2312500920016
:1066E000CF23B231A72B62080F39073A031DA72B1E
:1066F00021006808031DA72B20004B1ECB1D822BF9
:106700001030C906BE23B231CB1DA42B491A962BDB
:10671000A230250012020318962B21006808031DE1
:10672000962BCF23B2312500920AA42B2000491EBC
:10673000A42B21006808031DA42B250012080319AF
:10674000A32B9203A42BDB230C302100E8002000B4
:10675000490E890C890C01392400B300A43096310C
:106760000B26B23124003306031908000030200044
:10677000491B0130C700A4308631DD2E4B0C2400AC
:10678000B300B30C330C0139B400B40E20004B0835
:1067900024003406EF3934062000CB0008003D0009
:1067A0002108E0390C38A1000800620E890C890C20
:1067B0000339013A080022008E10E0303D00A105A7
:1067C0000800620E890C890C0339023A0800620E37
:1067D000890C890C0339033A0800E51FFF2B15309B
:1067E0005702031CF52B1430D70057082500A200D0
:1067F000A30120005708C7005530AA31402A671E60
:10680000ED2C073057020318512C60085706F03959
:106810005706E0005708C700B1308631DD26B33196
:106820005A302000C700B0308631DD26B331A731A1
:10683000E327B33103194F2C333096310B26B33194
:106840005A3A031D2A2C343096310B26B3312100DD
:10685000EF002D2C2100EF01EF0ABA310C22B331E9
:106860006108FC390138E10060080F39043A031966
:106870003F2CB5306111C7018631DD26B331B0310F
:10688000A420B3318631DD26B3312000B730C701F3
:10689000C70A8631DD26B331B7318C27B331AA312F
:1068A000432A0B3057020318862C08305702031C6A
:1068B000862CF930D7075708B0311520B33160085E
:1068C000B0317020B331E000600E890CB931AB21DA
:1068D000B331031C752C20006108B931AB21B331F1
:1068E000031C752C8731C427B33120005708C7001B
:1068F000B3308631DD26B3315A302000C700B230C4
:106900008631DD26B3312000B7309B2D0D30570284
:106910000318A22C0B305702031CA22CF530D7070A
:10692000570801396111031D6115003061190130EB
:10693000C700B5308631DD26B3315A302000C7009C
:10694000B430FD2B103057020318D32C0D305702F2
:10695000031CD32CF430D70761085706FC395706BF
:10696000E100600E890CB931AB21B331031CC22C9C
:1069700020006108B931AB21B331031CC22CBA31FC
:106980000C22B33120005708C700B7308631DD260E
:10699000B3315A302000C700B6308631DD26B3311E
:1069A0002000B3309B2D1230570203184F2C1030AB
:1069B0005702031C4F2CF030D707570801396012DB
:1069C000031D60165708C700B9308631DD26B33184
:1069D0005A302000C700B830FD2BE71EB82D083014
:1069E00057020318312D62085706F0395706E200A6
:1069F0005708C700C1308631DD26B3315A30200038
:106A0000C700C0308631DD26B331200062080F395F
:106A1000053A0319102D62080F39063A031D1E2D81
:106A2000A83096310B26B3312500120603191E2D0E
:106A3000B031A020B3318631DD26B33120006208A9
:106A40000F39073A031D262D250092012000620808
:106A50000F39023A03194F2C6208CF391038E2007F
:106A60009A2D0B3057020318662D08305702031C6D
:106A7000662DF930D707B0315820B33162082400B1
:106A80003906CF39B931FB21B331B931AB21B3313B
:106A9000031C552DBA310022B331B931AB21B331CA
:106AA000031C552D8731CA27B33120005708C70072
:106AB000C3308631DD26B3315A302000C700C230E2
:106AC0008631DD26B3312000C5309B2D0E305702B4
:106AD00003189E2D0B305702031C9E2DF630D7074E
:106AE0005708BA310522B3316208240039063F390C
:106AF000B931FB21B331B931AB21B331031C8B2D3B
:106B0000BA310022B331B931AB21B331031C8B2D23
:106B10008731BE27B33120005708C700C530863102
:106B2000DD26B3315A302000C700C4308631DD265F
:106B3000B3312000C330C701C70AFD2B1030570204
:106B400003184F2C0E305702031C4F2CF230D7077E
:106B5000570801396310031D63145708C700C73075
:106B60008631DD26B3315A302000C700C630FD2BF8
:106B7000BB31EE2B20268431E124B53140309631F3
:106B80000B26B5315A3A031DCA2D413096310B26DA
:106B9000B531CB2D04302100DE00423096310B267A
:106BA000B5315A3A031DE42D433096310B26B531E9
:106BB0002400C500C50D2000640824004506F939ED
:106BC00045062000E400E72DF9302000E4057F278A
:106BD000B5313C000F104926B531B827B53120003A
:106BE00092101026B5311C2627009115921592316E
:106BF0005422B531C726A2313C22B5314A262100A4
:106C0000921411141416003096310B26B531D93A6E
:106C100003190800D9302000C70000308631DD2E6E
:106C2000A33021009E00E0309F05833022009700B2
:106C3000553021009D0008008B1710160B17080017
:106C40008E1623008E169E31E1268C1623008C12A0
:106C500021000C1122000C1121000E1022000E1038
:106C600021008E1022008E1021000E1122000E1124
:106C700021008E1122008E1121000C1222000C1214
:106C800024000C1621000C108C1022000C148C1403
:106C90000800CA2F7011F0117012F0127017F11164
:106CA00071137211200060304C11E3115E1149160E
:106CB000CA114A124B12CB114A13CB104B104A1077
:106CC000CA10CC04A4307010F01068125110D1100A
:106CD000D1135210D21152115115611296310B2657
:106CE000B531FB27B531031C7C2E2000A430C70131
:106CF0008631DD26B5318D2EA43096310B26B53187
:106D00002200EF00EF0EEF0DEF0D200049082200EA
:106D10006F06BF396F062000C900A93096310B26D7
:106D2000B531FB27B531031C9C2E2000A930C701CB
:106D30008631DD26B531AC2EA93096310B26B53122
:106D40002200EF00EF0EEF0D20004A0822006F0630
:106D5000DF396F062000CA00A73096310B26B53107
:106D6000FB27B531031CB92E2000A730C70186319F
:106D7000DD2EA73096310B262200EF0020004908B7
:106D800022006F06FE396F062000C90008002000AF
:106D900055080339031DE82E733096310B26B531A3
:106DA0005A3A031DD92E763096310B26B531FF3E67
:106DB000DA2E05302100D9001F30FA01FA0A7A02D2
:106DC00003180800F527B531590881001F30DE2E61
:106DD00055080339023A031D182FFA010930FA0A3F
:106DE0007A020318F92EF527B531210059368100B2
:106DF000EE2E0930FA0013307A0203180A2FF52715
:106E0000B53121005908FF3E81001330FA0A7A0299
:106E1000031CFF2E1330FA001F307A0203180800FB
:106E2000F527B53121005908033E8100FA0A0C2FDD
:106E300055080339013A031D482F24000230C701C9
:106E4000C70AC800C900CA00CB000330CC00CD007F
:106E5000CE00CF000430D000D100D2000530D300E6
:106E6000D4000630D500D600D7000730D800D900AE
:106E7000DA000830DB00DC00DD000930DE00DF0076
:106E8000E0000A30E100E2000B30E300E40008001B
:106E900055080339033A031D0800FA010730FA0ABE
:106EA0007A020318582FF527B5318101810A4E2F38
:106EB0000730FA000E307A020318662FF527B53135
:106EC00081000E30FA0A7A02031C5E2F0E30FA009F
:106ED00019307A020318752FF527B5310330810078
:106EE0001930FA0A7A02031C6C2F04302400DF00E8
:106EF000E000E1000530E200E300E4000800A42720
:106F0000B531B027B5318C279631A526B531AA27E2
:106F1000B531D427B531DB2F2000921328001E1580
:106F2000FC309E0520005F1E9D2F60080F39043A3B
:106F3000031D9D2F033028009E04873028009E05E6
:106F4000A0309D009C0108008030970046309800DA
:106F50009501080051309B009C0199019A0108009D
:106F600092107E3028009700FF30960095010800AF
:106F7000BD27B531E127B531EA2F250097170F302E
:106F8000970417160C309F04FF30960095012000DF
:106F9000D21008002C00991719161F08FC39013867
:106FA0009F00980197010800413028009300940148
:106FB00091019201080021309A009B0198019901EA
:106FC0000800250093170F309304131603309F0415
:106FD00092010800260093170F30930413163030E7
:106FE00025009F042600920108007A08463E86008C
:106FF0000230870008002200EF0002306F02080014
:10700000FF3FFF3FFF3FFF3FFF3FFF3FFF3FFF3F90
:10701000FF3FFF3FFF3FFF3FFF3FFF3FFF3FFF3F80
:10702000FF3FFF3FFF3FFF3FFF3FFF3FFF3FFF3F70
:10703000FF3FFF3FFF3FFF3FFF3FFF3FFF3FFF3F60
:10704000FF3FFF3FFF3FFF3FFF3FFF3FFF3FFF3F50
:10705000FF3FFF3FFF3FFF3FFF3FFF3FFF3FFF3F40
:10706000FF3FFF3FFF3FFF3FFF3FFF3FFF3FFF3F30
:10707000FF3FFF3FFF3FFF3FFF3FFF3FFF3FFF3F20
:10708000FF3FFF3FFF3FFF3FFF3FFF3FFF3FFF3F10
:10709000FF3FFF3FFF3FFF3FFF3FFF3FFF3FFF3F00
:1070A000FF3FFF3FFF3FFF3FFF3FFF3FFF3FFF3FF0
:1070B000FF3FFF3FFF3FFF3FFF3FFF3FFF3FFF3FE0
:1070C000FF3FFF3FFF3FFF3FFF3FFF3FFF3FFF3FD0
:1070D000FF3FFF3FFF3FFF3FFF3FFF3FFF3FFF3FC0
:1070E000FF3FFF3FFF3FFF3FFF3FFF3FFF3FFF3FB0
:1070F000FF3FFF3FFF3FFF3FFF3FFF3FFF3FFF3FA0
:10710000FF3FFF3FFF3FFF3FFF3FFF3FFF3FFF3F8F
:10711000FF3FFF3FFF3FFF3FFF3FFF3FFF3FFF3F7F
:10712000FF3FFF3FFF3FFF3FFF3FFF3FFF3FFF3F6F
:10713000FF3FFF3FFF3FFF3FFF3FFF3FFF3FFF3F5F
:10714000FF3FFF3FFF3FFF3FFF3FFF3FFF3FFF3F4F
:10715000FF3FFF3FFF3FFF3FFF3FFF3FFF3FFF3F3F
:10716000FF3FFF3FFF3FFF3FFF3FFF3FFF3FFF3F2F
:10717000FF3FFF3FFF3FFF3FFF3FFF3FFF3FFF3F1F
:10718000FF3FFF3FFF3FFF3FFF3FFF3FFF3FFF3F0F
:10719000FF3FFF3FFF3FFF3FFF3FFF3FFF3FFF3FFF
:1071A0002300210874020318E12820005B08031D56
:1071B000E1285A080319DD28DA0321004C08031DD1
:1071C000CC01F119080021004C082000A000A10109
:1071D00074085A07A200A301A30D20082207A400E7
:1071E0002108233DA500803AA60080302602031D19
:1071F000FB28C1302402031CFF288F31B12FA0309F
:1072000020001E06031D0A290630F50074081E2101
:10721000B831192980301E06031D14290330F500EA
:1072200074081E21B831192960301E06031D1B2960
:10723000743674021C2974088F31A82FF600F801E7
:10724000750803193429F701F70AF51B2929F535C3
:107250002429F83575087602031C31297508F602D1
:107260007814F536F70B292978080800F3199029C6
:1072700020008C195B2928001208F500F601760819
:10728000F800220052087502F700031CF803780882
:10729000803AF90080307902031D502951087702A5
:1072A000031C5B29F016200095012800120822001B
:1072B000D2002800920120008C1D08000E3015021B
:1072C000031C080028009201200015082100C000BE
:1072D0000E304002031C72291F3040022330031875
:1072E00073297B2923304002031C7D29BF304002D3
:1072F00003187D290E302200D1002000530CF50028
:10730000F50C750C0F39013A031D8D295308073907
:10731000043A031D8D292200D1012200D201080068
:1073200020008C190800EC3028009200910173169F
:1073300021005A08031DDA030800073020005C050D
:107340002400B9000800CD302000C100CC30C200BC
:107350003D30C300080003392400B900023039026F
:10736000080020005C052400B900023A08007008FB
:1073700001392400B90020005C082400BA00013063
:10738000BA36BA363A05BB0039060800DC36DC36B8
:107390005C052400B9000800033020005C052400CF
:1073A000B900080001392400B90020005C0824005D
:1073B000BA0008002000E4136510E6136710E71018
:1073C000E5106511E5116512E5126513E513080076
:1073D0005C082400B900B936B93608002400B900A9
:1073E000B90C390C0139BA0008002000DC36DC3653
:1073F0005C080739080039062000E200620E080028
:107400002000620E890C890C08002400B900B90E16
:10741000B90DB90D20000800200060089F39203800
:10742000E0000800210046082400BA00BA36BA3647
:107430003A083906080020005D082400B900063427
:10744000560857040319282A0130D6020030D73BCA
:107450002200630864040319312A0130E30200307A
:10746000E43B200054193F2A023021003502D0307D
:107470000319340203183F2AB40A0319B50A711B11
:107480004C2A1E3022004802FF300319470203181D
:107490004C2AC70A0319C80A21002C082D04031915
:1074A000552A0130AC020030AD3B4F086E06031D7B
:1074B0005E2A7F304E0203185E2ACE0A220041085F
:1074C00042040319672A0130C1020030C23B210087
:1074D0002E082F040319702A0130AE020030AF3B92
:1074E0002200450846040319792A0130C5020030FC
:1074F000C63B430844040319812A0130C30200300B
:10750000C43B3D083E040319892A0130BD02003006
:10751000BE3B670868040319912A0130E702003076
:10752000E83B69086A040319992A0130E90200302E
:10753000EA3B21006808031DE80330083104031901
:10754000A82A7408031DA82A0130B0020030B13BFC
:1075500022003F0840040319B12A0130BF02003065
:10756000C03B21005D080319C62A2200610862049D
:107570000319BF2A0130E1020030E23BC62A210094
:10758000CD30DD032200E1000430E20022005F087C
:1075900060040319DC2A21002B0820005002031D7F
:1075A000D42A9F310A27BA310318DC2A013022007D
:1075B000DF020030E03B080022005D085E04031992
:1075C00008002000500821002B02031DEA2A9F31E9
:1075D000FB27BA310318080001302200DD02003019
:1075E000DE3B08001D3096310B26BA315A3A031D96
:1075F000FE2A1E3096310B26BA31132BE923BA31FD
:10760000031D042B0330132B56080339023A031DC4
:107610000D2B2100E501E50A152B56080339033A25
:10762000031D152B04302100E5001F3096310B2679
:10763000BA315A3A031D212B203096310B26BA312C
:10764000342BE923BA31031D272B0430342B560881
:107650000339023A031D2E2B0330342B560803390D
:10766000033A031D362B14302100E60021309631F9
:107670000B26BA315A3A031D422B223096310B2683
:10768000BA31532BE923BA31031D482B0530532B54
:1076900056080339023A0319462B56080339033AB0
:1076A000031D552B09302100E400233096310B26B1
:1076B000BA315A3A031D612B243096310B26BA3168
:1076C000742BE923BA31031D672B1E30742B560827
:1076D0000339023A031D6E2B1A30742B56080339F6
:1076E000033A031D762B20302100E300253096312C
:1076F0000B26BA315A3A031D822B263096310B26BF
:10770000BA31832B3D302200ED00273096310B2615
:10771000BA315A3A031D962B283096310B26BA31CE
:1077200096319426BA31DE23BA319B2B23002030C8
:10773000DF01E0004230E100B931A321BA31C523B5
:1077400096311D26BA31D223293096310B26BA3113
:107750005A3A031DBD2B2A3096310B26BA3121002F
:10776000E2002B3096310B26BA312100E1002C309B
:1077700096310B262100E000080008302100E200CD
:107780000430E100E001E00A080023005F08200067
:10779000C400230060082000C50023006108200009
:1077A000C600080041082300DF0020004208230033
:1077B000E000200043082300E10008002F08230018
:1077C000DF00200030082300E00020003108230003
:1077D0000800200056080339013A0800671D242CD0
:1077E0000B30570203180A2CB0315820BB315E0809
:1077F000240039060F3939062000DE005708C7007B
:10780000D5308631DD26BB315A302000C700D43058
:10781000AA31402A1030570203188F2C0E3057021D
:10782000031C8F2CF230D707570801396311031D51
:1078300063155708C700D3308631DD26BB315A3077
:107840002000C700D230082CE71D542C0730570207
:1078500003183A2C5F085706F0395706DF0057081F
:10786000C700D7308631DD26BB315A302000C70033
:10787000D630082C1030570203188F2C0E305702C8
:10788000031C8F2CF230D70757080139E311031D71
:10789000E3155708C700D9308631DD26BB315A3091
:1078A0002000C700D830082C661C742C803057028A
:1078B000031C5C2C7F30D700053057020318642C62
:1078C00004306116D700692C57352100DF002000F5
:1078D00061125708C7003D308631DD26BB315A3072
:1078E0002000C7003C30082CE61C912C05305702C4
:1078F000031C7C2C0430D70057082100DE00200038
:107900005708C70041308631DD26BB31B031A92090
:10791000BB318631DD26BB319631A526BB31AA317C
:10792000432A661DDB2C04305702031C992C0330BC
:10793000D70056085706FC395706D6005708C70027
:1079400047308631DD26BB315A302000C700463033
:107950008631DD26BB3192315422BB31B0317620E5
:10796000BB3196310B26BB31240039060319BA2CE2
:10797000FF30CD2C2000B0317620BB3196310B2664
:10798000BB3124003906031DD32C503096310B2611
:10799000BB315A3A0319D32C5A302000C70050305B
:1079A0008631DD26BB31A231A122BB31A331EE23CA
:1079B000BB31BF311C2FE61D312DFF30D7070430FE
:1079C0005702031CE52CD701D70A55085706FC3986
:1079D0005706D50003392400B900493096310B26EB
:1079E000BB312400390603190F2D20005508033937
:1079F000C70049308631DD26BB319731FC27BB31CA
:107A00008631DD26BB31B631C726BB31A331EE232B
:107A1000BB3180315620BB31A231A122BB31B03104
:107A20003420BB3196310B26BB31240039060319B3
:107A30001B2DFF302D2DB0313420BB3196310B265C
:107A4000BB3124003906031D8F2C543096310B2690
:107A5000BB315A3A03198F2C5A302000C7005430DA
:107A6000082CA93120292000D21F3B2D21000C1108
:107A70000E102000D21303305C052400B900023A36
:107A8000031D582D2000CD16F01C482D0130492D26
:107A900000302400B9002000541C502D0130512D1D
:107AA000003024003906031D5A2D2200D4015A2D1E
:107AB0002000CD12B931CC21BD31390B752D2000FC
:107AC0004D16F01C652D0130662D00302400B900E4
:107AD0002000541C6D2D01306E2D0030240039061D
:107AE0000319772D2200D401772D20004D1220009C
:107AF0004D1ECD1A7D2D2200D40AB931CC21BD31C5
:107B0000033A031D872D20004D172100CB0A2000CA
:107B10005C080339031D942D711121007130CA0ACC
:107B20002200BF000230C00020005C080339031DA2
:107B30009D2D2200D001D00A9F2D2200D0010C30B3
:107B40005406031DE22D0B30D40121004B02031C0F
:107B5000AB2D7115CD2D0B304B020318CD2D200010
:107B60000A30CD124D12711121004A02031CBA2DA8
:107B70000330C22D4A084B024B080318C52D0319C8
:107B8000C42D0230E700CD2D4B084A020318CD2D3D
:107B90004A080319CD2DE701E70ACA01CB01E22DFE
:107BA0002100C90120006030D901DB01CC04CB12D7
:107BB0002100C801F82DF11F7218F82D98311520F9
:107BC000BD31F82D20005D083F392400B900BA010D
:107BD0003A08003A0319ED2DDB2D3908003A031954
:107BE000F82D3E3A0319F82D013A0319D02DDB2D5B
:107BF000F11F7218942E7219942E2000541D942E89
:107C0000A03096310B26BD315A3A031D0E2EFF309F
:107C10002000C700A0308631DD26BD31A23096316C
:107C20000B26BD31003A03191B2E2000A230C701DC
:107C30008631DD26BD31BA311B22BD31B936890B03
:107C40001E2E3908031D962E2000E8192D2EB9315D
:107C5000B721BD31031D322E3F2EB931B721BD31C1
:107C6000031D3F2E200058359E314A26BD31AB0002
:107C700020005808D9002100D601D60AD7012000DB
:107C80005C082400B9000130B936B9363905BA00AC
:107C90002000680C2400BB00BB0C3B0C01393A06E9
:107CA000BC007006FE393C06F000F01C592E013075
:107CB0005A2E0030B900701C5F2E0130602E00304B
:107CC00039060319672EB0316420BD314C11701D87
:107CD000F01B742E2000B931E821BD31B9363908C6
:107CE0002000DB004C19DB0120005808A03E860074
:107CF000013087005B08A03E840001308500000849
:107D000001020318852EF216862EF212B931E821EF
:107D1000BD31B93639082100C8004808031D922E2C
:107D200020004C11AF315E2FAF316D2FBE31982E38
:107D3000BA311B22BE31B936890B9B2E3903AA31C9
:107D4000031D672ABE312000D41CFC2FB031B120A6
:107D5000BE31031DFC2FB931E821BE31BA311222E8
:107D6000BE31031DFC2F2000D410CA1BDD2EB931FB
:107D7000E821BE3139082300EF006F080319DB2E1C
:107D80003E306F020318DB2E6F082000D700731DF2
:107D9000CB2E3D30D70757082100EE009731EF2753
:107DA000BE318631DD26BE3120005708C7000230C3
:107DB0008631DD26BE31AF31592FB931E821BE31D0
:107DC00039082000D7009E31A226BE31031DEA2EBD
:107DD0003C30F72EB0319720BE31031DF12E7830A4
:107DE000F72E4C0E890C0339031DF82EB430D7073B
:107DF000E41F212F5708C70008308631DD26BE3129
:107E00005A302000C70007308631DD26BE31200001
:107E1000570896319426BE3197316B27BE31E70063
:107E2000B931A321BE3187312B27BE3196311D26B2
:107E3000BE3187314427BE3180315620BE31AA3150
:107E4000432A651C362F5708C7000A308631DD26C5
:107E5000BE315A302000C70009308631DD26BE31E0
:107E60002000570887318327BE311C2FE61F5B2F68
:107E70005708C7000E308631DD26BE315A3020004B
:107E8000C7000D308631DD26BE31200057089631FF
:107E90009426BE3197318127BE31E400B931A32148
:107EA000BE3197312E27BE3196311D26BE31973116
:107EB0005327BE311F2F671C762FFF30D707570877
:107EC000C70022005308803E8631DD26BE31803057
:107ED00096310B26BE315A3A03191C2F5A30200016
:107EE000C70080308631DD26BE311C2FE71CFE2FF7
:107EF0002A3057020318BA2F5708AF00FF30B001DD
:107F0000AF07031CB003A631C726BE312F082100DE
:107F1000A300200030082100A40020003108210027
:107F2000A50023082400A600210024082400A7009F
:107F3000210025082400A80084318C24BE312608A5
:107F40002000C70014308631DD26BE315A302000B3
:107F5000C70013308631DD26BE31B931A321BE31D1
:107F600097312127BE3196311D26BE3197314727E3
:107F7000BE311C2F2A305702031C1C2F5708AF009C
:107F8000D630B001AF07031CB003A631C726BE31FF
:107F90002F082100A000200030082100A1002000AF
:107FA00031082100A20020082400A6002100210899
:107FB0002400A700210022082400A80084318C247A
:107FC000BE3126082000C70012308631DD26BE31C2
:107FD0005A302000C70011308631DD26BE31B9315C
:107FE000A321BE3197311427BE3196311D26BE31F3
:107FF00097313B27BE311C2FAA315D2AA8311428A6
:020000040001F9
:08000E008C3FF635FF1FFF3F98
:10E00000D9005A003D00FF000100FF000000FF00A2
:10E010000D00FF001C005A000000FF000A00FF0076
:10E02000FF00FF00FF00FF00FF005A0003005A003E
:10E030000300FF00FF0000000000FF00FF00FF00E2
:10E04000FF00FF00FF00FF00FF00FF00FF00FF00D8
:10E05000FF00FF00FF00FF00FF00FF000200FF00C5
:10E060001E00FF004000FF000100FF000600FF004F
:10E070000000FF00FF0000005A0004005A000200E8
:10E08000FF000400FF000000FF00FF00FF00010090
:10E09000FF000000000000000000FF00FF00FF0084
:10E0A000FF00FF005A000C00FF000200FF00FF000D
:10E0B000FF00FF00FF00FF00FF00FF00FF00FF0068
:10E0C000FF00FF00FF00FF00FF00FF00FF00FF0058
:10E0D000FF00FF00FF00FF00FF00FF00FF00FF0048
:10E0E000FF00FF00FF00FF00FF00FF00FF00FF0038
:10E0F000FF00FF00FF00FF00FF00FF00FF000F0018
:10E10000FF00000000000000000000000000000010
:10E1100000000000000000000000000000000000FF
:10E1200000000000000000000000000000000000EF
:10E1300000000000000000000000000000000000DF
:10E14000FF000100000001000000000003000000CB
:10E15000FF000000FF00FF00FF00FF00FF00FF00C6
:10E16000FF000100FF000100FF000000FF000100B0
:10E17000FF000000FF00FF00FF00FF00FF00FF00A6
:10E18000FF000100FF000100FF000100FF00000090
:10E19000FF00FF00FF00FF00FF00FF00FF00FF0087
:10E1A000FF00FF00FF000000FF000100FF00010072
:10E1B000FF000000FF00FF00FF00FF00FF00FF0066
:10E1C000FF00FF00FF00FF00FF00FF00FF00FF0057
:10E1D000FF00FF00FF00FF00FF00FF00FF00FF0047
:10E1E000FF00FF00FF00FF00FF00FF00FF00FF0037
:10E1F000FF00FF00FF00FF00FF00FF00FF00FF0027
:080000006B050317002110013C
:00000001FF
